S31508001800A00A0020D9180008E7180008E9180008F7
S3150800181000000000000000000000000000000000BA
S315080018200000000000000000000000000119000888
S31508001830000000000000000003190008B93B00087A
S31508001840194C0008071900080719000807190008A5
S3150800185007190008071900080719000807190008DA
S31508001860071900089D290008071900080719000824
S3150800187007190008071900080719000807190008BA
S3150800188007190008000000000000000007190008FA
S3150800189000000000071900080719000807190008C2
S315080018A0000000000719000807190008414600084B
S315080018B007190008071900080719000800000000A2
S315080018C0EE11AA550348854600F006FD0048004774
S315080018D079790008A00A00200B4880F308880B488D
S315080018E080470B480047FEE704207146084202D0AD
S315080018F0EFF3098001E0EFF30880714605F0A8FED2
S31508001900FEE7FEE7FEE7FEE7A00A0020213E000804
S31508001910C518000830B50B460146002020220124D0
S3150800192009E00D46D5409D4205D31D469540491B05
S315080019302546954040191546521E002DF1DC30BD4E
S3150800194070B500242546002801DA01244042002902
S3150800195001DA01254942FFF7DDFFAC4200D04042DB
S31508001960002C00D0494270BD03460B439B0703D0A9
S3150800197009E008C9121F08C0042AFAD203E00B7846
S315080019800370401C491C521EF9D27047D2B201E0BE
S315080019900270401C491EFBD270470022F6E710B5BC
S315080019A013460A4604461946FFF7F0FF204610BDBF
S315080019B0F8B502464A40D40F42004B0052085B086D
S315080019C09A4202D20246084611464A0023D0C30D5F
S315080019D04A00DDB2120EAD1A202D35DA490201266B
S315080019E0490AF6058A19002C00D0524220214F1BBD
S315080019F01146B9402A411018C20D9A4221D0002C2E
S31508001A0017D0012D08DCDA05801AD20F8019D20703
S31508001A10DBB200F077FBF8BDDA05801A0123400037
S31508001A201B06C01880185A428018CA0F104349006E
S31508001A3007E04908C2071143DA05801A80194008E9
S31508001A40801800F057FBF8BD61000122511A001BEF
S31508001A50F7E70122D2075140AAE70122D2075040F0
S31508001A60A6E7024670B54A40D30FDB0740002DD0E3
S31508001A704A002AD0010E140E000212020919400A61
S31508001A80520A8418E50104465443000A120A2E0431
S31508001A905043A4194219200CC543AA18120C012553
S31508001AA0AD03521C521912047F39240400D0521C6B
S31508001AB0104301D44000491EC2B20C06C0092018C2
S31508001AC0401C4008802A02D003E0002070BD400870
S31508001AD04000002900DA0020184370BD70B50246A0
S31508001AE04A40D50F40004A00ED0740085208002832
S31508001AF014D0002A12D0C40DD30D41020120C0050E
S31508001B005202490A520AE41A091812187D349142F7
S31508001B1001D3641C00E04900002C01DA002070BDE6
S31508001B200023914201D3891A03434008490000283B
S31508001B30F7D100290AD0914202D10121C90705E04F
S31508001B40914201D2012101E00121C943E005C018F3
S31508001B50401900F0CFFA70BDF0B507460846584060
S31508001B6087B0C00F049048000E465900400849083F
S31508001B70BC1A884105D2384631461E4617460B46DA
S31508001B8002465800400810434CD0300D03904005DB
S31508001B905900400D490D0590401A0290402872DA06
S31508001BA018030121000B09050843019004980092C7
S31508001BB0002805D0019952420020884100920190E0
S31508001BC0029840210A1A0199009800F05FFA054622
S31508001BD00C466B4607CB00F07AFAC0197141039A96
S31508001BE00E0D0023D71756401A467A40164344D09E
S31508001BF0049A002A2DD0029A012A039A15DC1205A6
S31508001C00C01A914101263605001C7141D20F059E66
S31508001C10D2070093019202962A46234600F0B8FAA4
S31508001C2007B0F0BD38463146FAE71605224A0F4690
S31508001C30B218C01AB74101210905001C4F41001806
S31508001C407F41114618187941E20F10436D19644116
S31508001C5013E0E2076D0815436408C2071443039AA4
S31508001C6001261205C01A91413605001C7141CE079E
S31508001C70400830434908C01851412A46234600F017
S31508001C807AFACDE7FFE7049801224000C117121A35
S31508001C9000238B4104983146C417381AA141EEE750
S31508001CA030B40124E407634030BC55E730B401245E
S31508001CB0E407614030BC4FE70000E0FFF0B51FB411
S31508001CC088B00B990998002448400999C00F490023
S31508001CD049080991C0070B990090490049080B91DA
S31508001CE009990898A64608431CD00B990A980843F0
S31508001CF018D0099801244000420D4800410D099862
S31508001D0024050003000B204309900B980003000BE1
S31508001D1020430B9050181C49401800220190144685
S31508001D20104605E0002001460DB0F0BD032801DA93
S31508001D30034600E003239C46C11A0AAE0AE05F0088
S31508001D4008ADED5B4F00F75B7D430027AA187C4181
S31508001D50491C5B1E6145F2DD410004AB5A52210461
S31508001D60120C0A43240C401C0828DFDB0198029059
S31508001D700099704601910090059B049A0799069868
S31508001D8000F006FAD0E700000DFCFFFFF0B50C46A0
S31508001D905C4085B0E40FE40703944C000026640811
S31508001DA059009446490802460296224321D06246C3
S31508001DB00A431ED06200570D4A000E032303550D31
S31508001DC0012402462C492405781B1B0B360B4018A8
S31508001DD023432643614600901C46501AB44103D358
S31508001DE00098401C009002E0921800985B41002879
S31508001DF003DA0020014605B0F0BD002001210905DF
S31508001E000746864611E064461D46141BB54106D3AF
S31508001E106546521BB341744607430C43A646CD0795
S31508001E2040084908284392185B4105460D43EAD104
S31508001E301046184313D0604619465040714008436F
S31508001E4006D06046101AB34106D20122002306E0E6
S31508001E5000220123DB0702E00122D2435310009837
S31508001E6074460105381C6141029C039D00196941AD
S31508001E7000F081F9BFE70000FD030000C217C10F9B
S31508001E80504010B54018CA079623002100F03AF9C9
S31508001E9010BD10B500229623114600F033F910BD87
S31508001EA00EB5C217C10F5040CA0740180021054B8E
S31508001EB00293019200910A460B4600F069F903B0B5
S31508001EC000BD0000330400000EB50549029100214B
S31508001ED000910A460B46019100F05AF903B000BD7D
S31508001EE033040000C20F410040020123400ADB050B
S31508001EF0D207090EC0187F2901DA002070479629F3
S31508001F0003DC9623591AC84001E096398840002A0E
S31508001F10F4D040427047410040020122400AD205EF
S31508001F20090E80187F2901DA00207047962903DCFC
S31508001F309622511AC8407047963988407047000063
S31508001F404A0009030123090B1B051943094B10B560
S31508001F50520D9A4201DA002010BD064B34339A42DC
S31508001F6003DC9A1A00F0A2F810BD034951188840FC
S31508001F7010BD0000FF030000CDFBFFFFC20FD20714
S31508001F80400040080BD0C10D0723DB01C9184002E9
S31508001F900905400A1143C20840071143704700204B
S31508001FA00146704710B5002904DB0124E4074042C6
S31508001FB08C412146002B04DB1C460123DB075242D9
S31508001FC0A3418B4200D1824210BD0000CB0FDB0734
S31508001FD0490010B5490802460A4307D00A0D0724E6
S31508001FE00903E401090B121B002A01DC002010BDBD
S31508001FF0C900440F0C43C100E018D205801800F050
S3150800200079F810BD0122D207002800DB101A002932
S3150800201000DB511A814270470122D207002800DBF3
S31508002020101A002900DB511A88427047F0B51FB410
S315080020300646002082B005464024019100901BE028
S31508002040019922460F46304600F030F8049A059B5F
S31508002050801A994110D310461946224600F016F800
S31508002060361A8F410197224601200021009F00F071
S315080020700DF838184D4100902046641E0028DFDC14
S31508002080019B00982946324607B0F0BD10B5202AB4
S3150800209004DB0146203A9140002010BD91402023E0
S315080020A09C1A0346E3401943904010BD10B5202AF8
S315080020B004DB0846203AD040002110BD0B46D34029
S315080020C0D0402024A21A91400843194610BD10B5E5
S315080020D0202A06DBCB170846203A1041C1170B43C6
S315080020E006E00B461341D0402024A21A914008432B
S315080020F0194610BD002904DA401C490001D14008E0
S315080021004000704770B40024050C05D11024000463
S3150800211002D1002921D01124050E01D1000208346C
S31508002120050F01D10001241D850F01D18000A41CD3
S31508002130002801DB4000641C002908D020252E1B3E
S315080021400D46F540A14000D0012129430843010668
S315080021501B1B000ADB1D02D5002070BC7047DB057F
S31508002160181880180029F8DA401C4900F5D170BC07
S3150800217040084000704710B5002B08DA0024401CC0
S31508002180614192185B411A4301D14008400010BDD5
S31508002190F0B51FB482B005460C0003D0084602F01D
S315080021A0A7FD02E002F0A4FD203002460090214679
S315080021B02846FFF76BFF049B059A04460F4618430B
S315080021C01143084314D0184610431BD000984021E9
S315080021D00A1A18460599FFF769FF05460E46009A3A
S315080021E005990498FFF752FF084305D0012004E03B
S315080021F02046394607B0F0BD0020C11705430E43F7
S315080022002C43374300990E986305401A7905E40A6A
S3150800221000220C43FD0A0A3002D500200146E9E7F0
S315080022200105101969410C9C0D9D00196941FFF7BC
S31508002230A2FFDFE7FEB500231A461B1A8A4103DB15
S315080022400020014603B0F0BD4A000D0301212D0B05
S315080022500905520D0D43D10702D100186D41521ED2
S315080022605110FF31FF310131002704463E463846FA
S31508002270009701910246012100200905FFF716FF84
S31508002280C3197141F818324684468E464A4161465A
S315080022902846611A904104D36046241A9541764629
S315080022A01F46241900986D41401C00903428E1DD32
S315080022B0F91930467041091BA84103D20022D243BE
S315080022C0134601E00022134601980105381C7141A6
S315080022D0FFF751FFB6E70000064C0125064E05E05C
S315080022E0E36807CC2B430C3C98471034B442F7D329
S315080022F0FFF7ECFA749600089496000870B58C18E7
S315080023000578401C6B075B0F01D10378401C2A1126
S3150800231006D10278401C03E006780E70401C491C62
S315080023205B1EF9D12B0705D40023521E0DD40B7062
S31508002330491CFAE70378401CCB1A921C03E01D7867
S315080023400D70491C5B1C521EF9D5A142D8D300203A
S3150800235070BD000010B50446002C08D101210920E3
S31508002360C00600F0E7FD002000F0E6F852E0012C78
S3150800237005D102210920C00600F0DCFD4AE0022C46
S3150800238005D104210920C00600F0D4FD42E0032C43
S3150800239005D108210920C00600F0CCFD3AE0042C3E
S315080023A005D110210920C00600F0C4FD32E0052C35
S315080023B005D120210920C00600F0BCFD2AE0062C24
S315080023C005D140210920C00600F0B4FD22E0072C03
S315080023D005D180210920C00600F0ACFD1AE0082CC2
S315080023E004D101210D4800F0A5FD13E0092C04D104
S315080023F002210A4800F09EFD0CE00B2C04D11021A6
S31508002400064800F097FD05E00C2C03D1802103480F
S3150800241000F090FD204600F08FF810BD000400483B
S315080024207FB500200090019002900390002427E0D9
S3150800243000250CE0E800294940186100405AA1002F
S315080024406A4651584018A1005050681C85B2142D90
S31508002450F0DBA1006A4650581421FFF75BFA2821E1
S31508002460484361001E4A515A3C225143461864218A
S315080024703046FFF74FFA6100194A5052601C84B281
S31508002480042CD5DB1748807B002826D014484088C2
S315080024901549884203DC1248808888420ADD1148BB
S315080024A04038C07F002805D11049486005210D48ED
S315080024B04038C1770A4840880A2803DB08488088DC
S315080024C00A280ADA07484038C07F002805D1074994
S315080024D04860042103484038C1777FBDE8040020DE
S315080024E0740100202C040020E60F00000C020020D6
S315080024F000B587B001A800F0AFF80121480201F045
S31508002500CDF90020019070200290012080020390EE
S3150800251000200690059001A9064800F031F801212F
S31508002520044800F021F80121024800F011F807B02C
S3150800253000BD00000024014010B504460723002210
S315080025402146024800F038F810BD0000002401407A
S31508002550002904D0426801231A43426003E0426816
S315080025605208520042607047002904D08268082346
S315080025701A43826003E0826808239A4382607047A0
S3150800258042680B4B1A4042600B684A681A43436814
S315080025901A4342608268074B1A4082600B694A698F
S315080025A01A438B681A4383681A438260704700008F
S315080025B00FBCFFFF8FF1F9FFF0B504460D4616462E
S315080025C01F463F073F0F2B46082B0FD91B071B0F2C
S315080025D0083B606F9A000F21914088436067606FDF
S315080025E099003A468A40104360670BE0206F9A00CC
S315080025F00F21914088432067206F99003A468A4008
S3150800260010432067E0680121A9408843E060E0683C
S315080026100121A9400843E0600120800328400028E2
S3150800262003D0012000F020F807E00120C00328406D
S31508002630002802D0012000F017F8F0BD002905D0C7
S315080026408268FF2301331A43826004E08268FF230D
S3150800265001339A43826070470021016041608160BE
S315080026600173016141617047002806D0064949682F
S315080026700C221143044A516005E0034949680C22BB
S315080026809143014A516070470024014010B524481F
S315080026900078012834D10020214908702149088092
S315080026A012E02048008840001F49085A1F49098837
S315080026B0C9001F4A89181B4A1288520088521948AD
S315080026C00088401C17490880164800880428E8DB5B
S315080026D07E2002F0ADFA022000F02EF901211548FD
S315080026E0FFF7ACFF11480088401C104908800846CF
S315080026F00088142804DB0020088001200E49087091
S315080027000D480078002806D0FFF78AFE00200A49FF
S31508002710087000F059FC7E2002F08AFA10BD00000D
S31508002720840100209E010020B0040020A0010020A2
S31508002730E8040020002401407C010020FFB583B096
S315080027400C46029400200190002726E000261CE093
S31508002750721C039951430846791CFFF7DBF80546B6
S31508002760A54201D9281B00E0601B05460298A8422D
S3150800277004D90295059806700698077002980028ED
S3150800278002D10120019002E0761C402EE0D300BF62
S315080027900198002800D002E07F1C042FD6D300BF82
S315080027A0029807B0F0BD000000BF00BF00BF00BF21
S315080027B000BFBFF34F8F00BF00BF00BF06480749E1
S315080027C0C86000BF00BF00BFBFF34F8F00BF00BF88
S315080027D000BF00BF00BFFDE70400FA0500ED00E0FA
S315080027E010B500F001F810BD10B523480078002890
S315080027F017D1224801F0DAF801283CD11F480078A1
S31508002800002838DD1D480078402834DC01F0ECFE4D
S315080028101B490860012018490870002019490870EA
S3150800282029E0164A17490978491C501801F0BEF8DC
S31508002830012816D113480078401C124908700F4821
S3150800284000780978884216D100200B4908700B4891
S315080028504078FF280FD10B48007802280BD1FFF7E4
S31508002860A3FF01F0C1FE064909686431884202D90E
S3150800287000200149087010BD490100206C040020A1
S315080028804C0100204801002010B586B004460121FD
S31508002890880301F003F80121480400F0DFFF012254
S315080028A00921C80600F031FB01220A210920C006C9
S315080028B000F02BFB01A801F098FF0194302168462F
S315080028C0018100214181818101821821C18101A9EB
S315080028D0184801F047FF0121164801F020FF05A816
S315080028E000F069FB01214902684681820121817550
S315080028F01821C17505A90920C00600F0B9FA0121F9
S315080029008902684681824821C17505A90920C00641
S3150800291000F0AEFA1B2168460170032141700121BF
S31508002920817000F067FF01220221024801F00FFFC3
S3150800293006B010BD0038014001B506490098086088
S3150800294002E07E2002F074F9024800680028F8D1F7
S3150800295008BD000054010020014600220E4B1A61F2
S31508002960CA005A6100229A6105221A6100BF0A4A02
S315080029701069C207D20F002A04D0012212040240AD
S31508002980002AF4D0044A126952085200024B1A610E
S3150800299000229A617047000000E000E010B50021AF
S315080029A00448FFF74BFE022000F04AF801200249CE
S315080029B0087010BD002401408401002000B589B0CC
S315080029C00121084600F04AFF1A4800F045F801A818
S315080029D000F08EF8184801901848029000216846C1
S315080029E001730420049068460175802141754900E9
S315080029F0C182890001832021817609028183002111
S31508002A00C183018401A90B4800F04CF8012109484B
S31508002A1000F01CF801220221064800F039F80921C5
S31508002A2068460170022141700121817000F0E2FEC2
S31508002A3009B000BD0800024000240140B00400208F
S31508002A4001494860704700000000024002685208C9
S31508002A5052000A430260704710B5044620684008D1
S31508002A6040002060002020606060A060E060E1B265
S31508002A70084608380521FEF74DFF01460F20884015
S31508002A800249496808430149486010BD00000240F0
S31508002A90002A03D003680B43036002E003688B43F4
S31508002AA00360704710B50A7A8B7D1A430B7C1A436C
S31508002AB04B7C1A434B8A1A438B8A1A430B8B1A434D
S31508002AC04B8B1A430368094C23401A430260026879
S31508002AD00123DB039A438B8B1A430260CA68426060
S31508002AE00A6882604A68C26010BD00000F80FFFF56
S31508002AF00021016041600172C16001744174418224
S31508002B0081828175018341838183704770B506464A
S31508002B100C4621460A4800F04BF90546002D01D11E
S31508002B20401E70BD0648854202D10648051B00E0D6
S31508002B302D1B224629463046FEF716FF2046F0E7AB
S31508002B4000F4000800FC000870B506460C4621464D
S31508002B500A4800F02DF90546002D01D1401E70BD2A
S31508002B600648854202D10648051B00E02D1B224671
S31508002B7029463046FEF7F8FE2046F0E700A0000892
S31508002B8000A8000870B506460C4621460A4800F01B
S31508002B900FF90546002D01D1401E70BD0648854235
S31508002BA002D10648051B00E02D1B22462946304661
S31508002BB0FEF7DAFE2046F0E700B0000800B8000885
S31508002BC070B505460C4622460249284600F0B1F87B
S31508002BD0204670BD00F4000870B505460C4622462E
S31508002BE00249284600F0A5F8204670BD00A0000856
S31508002BF010B50446084800690221084306490861D9
S31508002C0008464461006940210843034908610348AE
S31508002C1000F00EF910BD000000200240FF0F000072
S31508002C200C48C068C007C00F002801D001207047B3
S31508002C300848C06804210840002801D00220F6E7A9
S31508002C400448C06810210840002801D00320EEE798
S31508002C500420ECE70020024003480069802108436D
S31508002C6001490861704700000020024030B504465B
S31508002C700D46054800690121084303490861258076
S31508002C800F2000F0D5F830BD0020024010B57E2098
S31508002C9001F0CEFF064800F00FF87E2001F0C8FFCD
S31508002CA0044800F009F87E2001F0C2FF10BD0000BC
S31508002CB000F4000800A0000810B5044600F0ACF8BF
S31508002CC02046FFF795FFFFF7C7FF10BD70B503460F
S31508002CD00125002208E050001C5A0748844201D00A
S31508002CE0002506E0501C82B2CE0F76187610964262
S31508002CF0F1DC00BF284670BDFFFF0000F8B50546A9
S31508002D000E46144600F088F87E2001F091FF002751
S31508002D1007E029883046FFF7A9FFB61CAD1C781CCA
S31508002D2087B2E10F09194910B942F2DCFFF794FF9F
S31508002D30F8BDF8B507460C4615462946204600F064
S31508002D4037F80646002E0DD12046FFF7B5FF0120BD
S31508002D5080022018FFF7B0FF2A4621463846FFF7BB
S31508002D60CDFF24E0012080022018401BB0420AD182
S31508002D70012080022018FFF79FFF2A463146384671
S31508002D80FFF7BCFF13E00120C0022018401BB04229
S31508002D9008D12046FFF790FF2A4631463846FFF706
S31508002DA0ADFF04E02A4631463846FFF7A7FFF8BDCF
S31508002DB0F8B505460E462F46E807C00F002801D08D
S31508002DC000BFFEE731460120C002FEF7B9FD002923
S31508002DD001D000BFFEE700240BE0204670434719E8
S31508002DE031463846FFF772FF012800D108E0601C1B
S31508002DF084B231460120C002FEF7A2FDA042ECDCF7
S31508002E0000BF31460120C002FEF79AFDA04200D15C
S31508002E1000273846F8BD00000248034948600348C1
S31508002E20486070472301674500200240AB89EFCD13
S31508002E3010B5024600BFFFF7F3FE0346521EFF24F5
S31508002E4000E0641E002CFCD1012B01D1002AF2D12E
S31508002E500648006977218843044908613420C86018
S31508002E60002A01D1052010BD1846FCE700200240C3
S31508002E70F8B50246CD782F073F0FCD781026354096
S31508002E80002D01D08D782F431446002011E08506C9
S31508002E902B0E0D88012686403540002D07D0256863
S31508002EA00F269E40B5433E469E4035432560451C49
S31508002EB0E8B20828EBDB141D0D882D1200950020BA
S31508002EC011E085062B0E01258540009E3540002D14
S31508002ED007D025680F269E40B5433E469E4035439B
S31508002EE02560451CE8B20828EBDBCD78282D04D1EF
S31508002EF055690E883543556106E0CD78482D03D1CE
S31508002F0015690E8835431561F8BD70B54D07EB0E8A
S31508002F10082902DA0546203501E0054624352C46FF
S31508002F200F269E402568B54316469E4035432560C4
S31508002F3070BD000038B504460D460920C006844217
S31508002F4003D10121480400F089FC1148844203D1C9
S31508002F500121000200F082FC0E48844203D10121BF
S31508002F60000200F07BFC0C48844203D101210805CD
S31508002F7000F074FC684600F01EF8684605800121DA
S31508002F8081700021C17069462046FFF771FF38BD80
S31508002F900004004800080048000C004802469068F3
S31508002FA00840002801D0012070470020FCE7416155
S31508002FB07047016170470021C94301800221817071
S31508002FC00421C1707047000000B591B000200F9031
S31508002FD00E900D900C907E2001F02AFE0020109095
S31508002FE01FE010984000FE49085A0590FEF751FF69
S31508002FF0FC490690FEF772FD0790FEF7BFFF002218
S31508003000F94B09910890FEF759FE0B910A90FEF7C5
S31508003010DDFF10998900F54A50501098401C80B27F
S31508003020109010980428DCDBF0488068F049069078
S31508003030FEF754FD0790FEF7A1FFEE4AEE4B099105
S315080030400890FEF733FE0B910A90FEF7BFFF0F902C
S31508003050E6484068E6490690FEF740FD0790FEF709
S315080030608DFFE44AE44B09910890FEF71FFE0B9189
S315080030700A90FEF7ABFF0E900F98FEF77FFF00222F
S31508003080D94B05910490FEF711FE09910890DB488B
S315080030900F99FEF7E6FC0590FEF770FF079106907C
S315080030A0099B089AFEF772FE0B910A90FEF78EFFAF
S315080030B0D34908600E98FEF761FF0022CA4B0591B6
S315080030C00490FEF7F3FD09910890CC480E99FEF797
S315080030D0C8FC0590FEF752FF07910690099B089ACF
S315080030E0FEF754FE0B910A90FEF770FFC54908607B
S315080030F0C548008D322830DAC448408B0190FEF767
S31508003100E3FEC34AC34B03910290FEF7D7FD0022A4
S31508003110C14B05910490FEF739FE09910890BB480A
S31508003120408B0290FEF7B5FEBC490390FEF7D6FC2D
S315080031300490B34801680498FEF78FFC0590FEF7E3
S315080031401DFF07910690099B089AFEF71FFE0B9133
S315080031500A90FEF73BFF0D905CE0AB48008DBE2859
S315080031602CDAAA48408B0690FEF793FE0890A748EB
S31508003170808B0590FEF78DFEA9490690FEF7AEFCFA
S3150800318007900899FEF76DFCA4490990FEF7A6FC7E
S315080031900B909E48408B0790FEF77BFE9F49089050
S315080031A0FEF79CFC0990964801680998FEF755FCBD
S315080031B00A900B99FEF792FC0D902BE09348408BF2
S315080031C00690FEF766FE08909048008C0590FEF77C
S315080031D060FE93490690FEF781FC07900899FEF772
S315080031E040FC8E490990FEF779FC0B908748408B86
S315080031F00790FEF74EFE89490890FEF76FFC099086
S315080032007F4801680998FEF728FC0A900B99FEF793
S3150800321065FC0D907C48408D322830DA7B48008B5F
S315080032200190FEF751FE7A4A7A4B03910290FEF717
S3150800323045FD0022784B05910490FEF7A7FD0991FC
S3150800324008907248008B0290FEF723FE734903909C
S31508003250FEF744FC04906B4801680498FEF7FDFBF2
S315080032600590FEF78BFE07910690099B089AFEF7D4
S315080032708DFD0B910A90FEF7A9FE0C905CE0624862
S31508003280408DBE282CDA6148008B0690FEF701FEB9
S3150800329008905E48C08B0590FEF7FBFD60490690D6
S315080032A0FEF71CFC07900899FEF7DBFB5B490990C3
S315080032B0FEF714FC0B905548008B0790FEF7E9FDC6
S315080032C056490890FEF70AFC09904E480168099885
S315080032D0FEF7C3FB0A900B99FEF700FC0C902BE057
S315080032E04A48008B0690FEF7D4FD08904748408C64
S315080032F00590FEF7CEFD4A490690FEF7EFFB0790CC
S315080033000899FEF7AEFB45490990FEF7E7FB0B90D7
S315080033103E48008B0790FEF7BCFD40490890FEF733
S31508003320DDFB0990374801680998FEF796FB0A9075
S315080033300B99FEF7D3FB0C903A480D99FEF738FB2C
S315080033400B90FEF7E8FD3849086036480C99FEF7F9
S315080033502FFB0B90FEF7DFFD344908602A48008DE5
S31508003360314909684018C003010C27480185408D7A
S315080033702E4909684018C003010C234841851B489B
S31508003380C0682B490A90FEF76CFB0B90FEF7C3FD4D
S3150800339081B21D480187FF38C1380088FF21F53101
S315080033A0884276DD00201949683908800F48006888
S315080033B00990FEF7E3FD1F4A1F4B0B910A90FEF793
S315080033C0F1FD56D2094800680990FEF7D7FD1B4A59
S315080033D01B4B0B910A90FEF7E5FD45D2402131E0E3
S315080033E07401002000F07F4500000840D804002042
S315080033F00000404125068195438BD43F0000484391
S315080034008C01002090010020CC03002074020020CB
S31508003410091B9E5E29CB703F00408F4000007A440E
S31508003420002474490000C841940100209801002036
S315080034300000C842736891ED7C3FDD3F9CC420B014
S315080034407268D13F2B48FFF7A9FD00280CD12A48FE
S31508003450407F012808D12848C07F002804D1274981
S31508003460486006212448C177012023494031087164
S3150800347014E02348006823490B90FEF7CDFD0DD2D2
S315080034801D484030807B002804D11B494031087113
S3150800349004E02CE0012018494031087118480068FA
S315080034A019490B90FEF7B8FD04D2012112484030A5
S315080034B0417103E000211048403041710E48403008
S315080034C0007900280ED10C48407F012804D101025A
S315080034D00848FFF76CFD0AE0FF2101310548FFF7B0
S315080034E068FD04E0FF2101310248FFF762FD11B0D3
S315080034F000BD000000040048EC0300200C02002078
S31508003500D80400206F12233F333313400148806AE2
S3150800351070470000C0F7FF1F0148006870470000A9
S3150800352058010020034800680349097840180149F2
S3150800353008607047580100206001002008B5012185
S31508003540480400F08BF90121880400F087F96846E1
S31508003550FFF731FD0121C903684601804821C17082
S3150800356069460920C006FFF783FC6846FFF723FD76
S3150800357001210903684601804821C170694609206E
S31508003580C006FFF775FC6846FFF715FD402168463B
S3150800359001800421C17069460148FFF769FC08BD2E
S315080035A00004004810B50121C9030920C006FFF729
S315080035B0F5FC002841D16A488078002831D168484E
S315080035C02038407F012829D165482030807B002893
S315080035D024D164480078401C62490870084600787F
S315080035E005281BDB0020087004215F48FFF7E1FC73
S315080035F05B4898384089002807D15C485C49486090
S31508003600012157489838418106E00020584948600A
S31508003610002153489838418101F02AFB012150487E
S31508003620817054480078002810D10120514908704B
S3150800363001214B482038817708E000204D49087061
S315080036400021474820388177203081704848C06873
S31508003650464988427DD900204549C860002140482E
S31508003660203881774030807B00286BD108213E487E
S31508003670FFF79FFC3A4898384088032869DA3848A3
S3150800368098384089002864D135484038408D8228CA
S3150800369010DA33482030407900280BD130482038DA
S315080036A0407F012855D12E492031887300203049A2
S315080036B048604EE02A482038407F012802D1002081
S315080036C02B49486026484038408D822830DB2A48F6
S315080036D040882A49884203DC2748808888420ADDD0
S315080036E01F482038C07F002805D121494860052198
S315080036F01B482038C177204840880A2803DB1E4823
S3150800370080880A280ADA16482038C07F002805D19A
S3150800371017494860042112482038C17710482038D4
S31508003720C07F002815D102210D482038C17710E046
S315080037300B482030407901280BD101210848203850
S31508003740C17706E000200A4948600021044820386D
S3150800375041777E2001F06CFA01482038807F10BD41
S315080037600C040020C400002000040048DC0500000A
S315080037700C020020A201002074010020E60F0000C0
S3150800378008B50121480400F069F80121880400F011
S3150800379065F86846FFF70FFCFF210E316846018081
S315080037A0012181701021C17069461148FFF760FB3D
S315080037B0B62168460180012181701021C1706946D1
S315080037C00920C006FFF754FB10210920C006FFF7A1
S315080037D0EEFB80210920C006FFF7E9FB012104481A
S315080037E0FFF7E5FB08210248FFF7E3FB08BD0000E9
S315080037F0000400488178002925D0174903221202BF
S315080038008918027892109200895802789207D30E86
S31508003810FF229A40914342789207120E03789B073B
S31508003820DB0E9A4011430C4A03231B02D218037875
S315080038309B109B00D1500178CA06D20E01219140F7
S31508003840054A116007E00178CA06D20E01219140A7
S31508003850014A80321160704700E100E0002905D076
S31508003860054A52690243044B5A6104E0024A526906
S315080038708243014B5A61704700100240002905D067
S31508003880054AD2690243044BDA6104E0024AD26966
S315080038908243014BDA61704700100240002905D0C7
S315080038A0054A92690243044B9A6104E0024A926906
S315080038B08243014B9A6170470010024010B500F030
S315080038C031F804494968F02211400909024A515C55
S315080038D0C84010BD001002402201002010B5FFF7B5
S315080038E0EDFF05494968072212021140090A034AF1
S315080038F0515CC84010BD00000010024022010020A3
S3150800390010B5FFF7DBFF054949680722D2021140C7
S31508003910C90A034A515CC84010BD000000100240A5
S3150800392022010020F8B51E4840680C2108400428EA
S3150800393002D008282ED101E01A4C2DE01848403054
S315080039400069C007C00F00280AD015484030006932
S3150800395002210840002801D0134802E0114800E07F
S31508003960104807460E4840300069FF210904084000
S31508003970000C451C0A484030006907210902084026
S31508003980000A461C3946694308463146FDF7C2FF18
S31508003990044601E0034C00BF00BF2046F8BD000006
S315080039A00010024000127A0000093D0070B5044676
S315080039B000250221074800F0B8FE002808D005486F
S315080039C000F00CFF20700221024800F0A6FE012537
S315080039D0284670BD0038014010B500F001F810BD4A
S315080039E000B585B06248006801210843604908604F
S315080039F000BF5F480068022108400028F9D05D48EA
S31508003A005D4908605D480068102108435B49086005
S31508003A1008460068C008C000086057490968481E7B
S31508003A205749FDF777FF04905448006804994907F9
S31508003A30490F0843514908604D48406851490840B4
S31508003A404B49486008464068902108434849486001
S31508003A50084640684860484800684649884207D989
S31508003A6043484068052109020843414948600BE07C
S31508003A70414800684449884206D93D4840680121C2
S31508003A80890208433A4948606B4601AA3A480168E0
S31508003A903E48FEF753FE36484030006980088000ED
S31508003AA0334940310861084600694008400008610A
S31508003AB0684600784007400F02906846007940063D
S31508003AC0400E03902A48C069890508432849C861F9
S31508003AD02748403000692E49084025494031086189
S31508003AE003980004029909020843214940310969EB
S31508003AF008431F49403108611D480068012109062D
S31508003B0008431B49086000E000BF19480068012106
S31508003B10490608400028F7D0154840688008800004
S31508003B20134948600846406802210843104948601E
S31508003B3000E000BF0E4840680C2108400828F8D16C
S31508003B400120FEF709FF0A48406810218843084902
S31508003B5048600120FEF700FF054840688021884339
S31508003B60034948600120FEF7F7FE05B000BD0000D6
S31508003B700010024000A24A0434010020002002403E
S31508003B8000366E010FC0FFFF0051250200127A00B1
S31508003B90FFF800FF042806D10649096904221143E3
S31508003BA0044A116105E00349096904229143014A5F
S31508003BB01161704700E000E010B5FFF7B3FC9148CB
S31508003BC00088401C8F49088008464068401C4860A9
S31508003BD08D480088401C8C4908808C48006800285D
S31508003BE004D08A480068401E884908608848807F53
S31508003BF0012805D18348C068401C8249C86002E094
S31508003C0000208049C86082484030807A012805D162
S31508003C107C484069401C7B49486102E0002079499C
S31508003C2048617B4820300078012805D17548006C2A
S31508003C30401C7449086402E000207249086471490E
S31508003C4048680A21FDF766FE002923D1704820300E
S31508003C50C17F807F814208DD6D482030807F401C0F
S31508003C60C1B26B482030817714E069482030C17FA3
S31508003C70807F814200D10DE065482030C17F807F7A
S31508003C80814207DA62482030807F401EC1B2604810
S31508003C90203081775E484030807B022804D05C481B
S31508003CA04030807B032804D15648806B401C554918
S31508003CB0886357484030407800280AD15448403035
S31508003CC0807B042805D14F48806C401C4D49886488
S31508003CD002E000204B4988644D484030807B00282C
S31508003CE003D148490865C86428E049482030C078A7
S31508003CF0012805D14348006D401C4249086502E089
S31508003D00002040490865424820300079012812D130
S31508003D103C48C06C401C3B49C8643D4840308078EC
S31508003D20002804D108468068401C886006E0002008
S31508003D303449886002E000203249C8643448807EED
S31508003D4004280AD12F48406D3249884208D22D48A6
S31508003D50406D401C2B49486502E00020294948650A
S31508003D60012109030920C006FFF718F9002813D016
S31508003D7027484030007900280ED12548407F012881
S31508003D800AD12048806D2449884208D21D48806D92
S31508003D90401C1C49886502E000201A4988651C48B1
S31508003DA04030807901280AD11648C06D1B498842DF
S31508003DB008D21448C06D401C1249C86502E00020AC
S31508003DC01049C86512484030007A012805D10D48C7
S31508003DD0006E401C0B49086602E000200949086687
S31508003DE00B484030407A012805D10648406E401CF1
S31508003DF00449486602E00020024948667E2000F031
S31508003E0017FF10BD0C0200205001002054010020AD
S31508003E10EC03002050C30000881300007017000050
S31508003E2010B5164800680121084314490860084679
S31508003E304068134908401149486008460068114916
S31508003E4008400E490860084600680121890488432D
S31508003E500A49086008464068C32109048843074997
S31508003E6048600846006808490840044908609F20D9
S31508003E7000048860FFF7B0FD10BD00000010024086
S31508003E800CC0FFF8FFFFF6FEFFFF8F0008B5012103
S31508003E904804FFF7E3FC022201210920C006FFF7C8
S31508003EA034F80221684601801821C1700121817009
S31508003EB069460920C006FEF7DBFF01214804FFF723
S31508003EC0CDFC022211460920C006FFF71EF8042180
S31508003ED0684601801821C170012181706946092050
S31508003EE0C006FEF7C5FF08BD30B587B004460D46C7
S31508003EF001210846FFF7C2FC04A800F033F905942F
S31508003F0068460582002101838176817404A901200F
S31508003F10800700F0F1F8684600F0D2F8602168469C
S31508003F20017001214170002001900021684601724C
S31508003F3069460120800700F057F869460120800786
S31508003F4000F08AF80821C80600F07EF80821C8069D
S31508003F5000F0B0F84021080600F038F840210806BD
S31508003F6000F03CF80121880700F00AF801218807CB
S31508003F7000F01EF80121880700F00EF807B030BDE2
S31508003F80002904D0026880231A43026003E002680D
S31508003F9080239A4302607047002904D002680123EF
S31508003FA01A43026003E00268520852000260704732
S31508003FB0002905D0426C0123DB031A43426404E05E
S31508003FC0426C0123DB039A434264704782690723E4
S31508003FD01B039A430B021A4382617047C269702316
S31508003FE09A430A43C261704710B5826907231B03C7
S31508003FF09A430B781B021A4382610A7A12014B789C
S315080040001B011A43036A3024A3431A4302624A680F
S3150800401082630C4A904213D14A7A12018B781B01AB
S315080040201A43036AC024A3431A4302624A899200C8
S315080040308B899B001A4343682401A3431A434260B1
S3150800404010BD0000002C014082690123DB029A435F
S315080040500B021A438261704710B5C26970239A43EE
S315080040600B781A43C2610A7A12024B781B021A436A
S31508004070036A03242402A3431A4302624A68C263FA
S315080040800B4A904213D14A7A12028B781B021A43C2
S31508004090036AA400A3431A4302624A8912018B8960
S315080040A01B011A434368A400A3431A43426010BD88
S315080040B0002C0140C26908239A430A43C26170472B
S315080040C00021017041708170416001724172418125
S315080040D08181704701229207904201D1816301E0F4
S315080040E08AB28263704701229207904201D1C16366
S315080040F001E08AB2C2637047026803231B029A432F
S315080041000B891A430260134A904206D0012292078D
S31508004110904202D0104A904205D1026870239A4311
S315080041208B781A4302600B4A904205D00B4A90429C
S3150800413002D00B4A904205D1026B120A12028B7A00
S315080041401A4302634A68C2620A888262012242618D
S3150800415070470000002C0140000400400044014064
S31508004160004801400021C9434160002101800181C6
S31508004170817081727047000010B50024FA48807A71
S3150800418000280FD1F9484068F9490968401AF949E1
S3150800419088420BD90021F448403841770020F2497B
S315080041A0887303E0F1484068F1490860EE48C07931
S315080041B0030000F0B4FD050478F1EFEEED00EA49DE
S315080041C020398A8BE9494868B32104F071FE044610
S315080041D0E5482038408B912805DA0F220121002076
S315080041E002F02EF904E000220121104602F028F917
S315080041F0DD482038808BB42809D0DB482038808BEE
S31508004200B32804D0D8482038808BB52813D1D6488F
S315080042106038408DD8490988884208D00020D2499C
S31508004220487208466038408DD349088006E0012068
S31508004230CD49487202E00020CB494872CB48406E0F
S31508004240CE49884226D9C8482038408B801ECC499A
S315080042500988884216DCC4482038408B801CC84927
S31508004260098888420EDBC6480088A5280FDB02F0BD
S315080042702FFE0120BC49C8710020BC494866C149C7
S31508004280087004E0B8482038408BBD4908800020F3
S31508004290B64948660020BC490870224601210846EE
S315080042A002F0CEF897E1B04920390A8BAF49486841
S315080042B0B32104F0FDFD044600220121084602F060
S315080042C0BFF8A9482038008BB42809D0A64820385A
S315080042D0008BB32804D0A4482038008BB52813D106
S315080042E0A1486038008DA4490988884208D0002072
S315080042F09D49487208466038008D9F49088006E047
S3150800430001209949487202E0002097494872974867
S31508004310406E9A49884222D993482038408B801E9D
S3150800432097490988884212DC8F482038408B801CC0
S315080043309349098888420ADB02F062FE02208A490C
S31508004340C8710020894948668E49087004E0864885
S315080043502038408B8A4908800020844948668A4864
S31508004360007800280ED180482038808B822805DD09
S3150800437000220121104602F063F808E00120824974
S31508004380087004E022460121002002F059F822E1D3
S3150800439020E107E16BE0FFE7734920398A8B73490F
S315080043A04868E52104F084FD0446002201211046F0
S315080043B002F046F86C482038808BE62809D06A480F
S315080043C02038808BE52804D067482038808BE7287A
S315080043D013D165486038408D67490988884208D0F6
S315080043E000206149487208466038408D6249088055
S315080043F006E001215C48417202E000215A484172F8
S315080044005A48406E5D49884228D957482038408B1B
S31508004410801E5B490988884218DC53482038408B3F
S31508004420801C57490988884210DB55480088D228DD
S3150800443011DB02F07DFE03204B49C87102F014FD22
S3150800444000204A4948664F49087004E04648203823
S31508004450408B4B49088000204449486600204B4958
S31508004460087022460121084601F0EAFFB3E03E49FA
S3150800447020390A8B3D494868E52104F019FD0446B0
S3150800448000220121084601F0DBFF37482038008B5F
S31508004490E6280BD034482038008BFF212C3188427F
S315080044A004D031482038008BE72813D12E486038CD
S315080044B0008D31490988884208D000202A49487267
S315080044C008466038008D2C49088006E001202649F8
S315080044D0487202E00020244948722448406E274961
S315080044E0884231D920482038408B801E24490988C3
S315080044F0884221DC1C482038408B801C20490988CA
S31508004500884219DB1E480088C3281ADB1C48008825
S31508004510D22816DA02F0A4FE04201349C87102F064
S31508004520A3FC0122FE21572003F0CBFC00200F49F3
S3150800453048661449087004E00B482038408B104937
S31508004540088000200949486610480078002823D1C9
S3150800455005482038408BC8281ADD0022012110465C
S3150800456001F06EFF1DE000002C0400200C02002064
S3150800457010010020C409000016010020DC05000017
S315080045800C010020F8000020180100201901002065
S3150800459001201249087004E022460121002001F09A
S315080045A04FFF18E00E494868FF21F531FDF7B2F9CB
S315080045B000290ED100200A4948660A494885002282
S315080045C00121104601F03CFF00220121084601F0B6
S315080045D037FF00E000BF00BF10BD00001901002032
S315080045E00C0200203C04002010B5FEF795FF10BD14
S315080045F070B5FFF763F905467D21C900FDF78AF90D
S315080046000446601E0C49884200D90CE0601E0B491E
S3150800461048610321081F00F091FB002007498861C3
S315080046200720086100BF0420FFF7B4FA0021481EDE
S3150800463000F084FB70BD0000FFFFFF0000E000E013
S3150800464010B50221134800F079F8002820D0114847
S3150800465000F0C4F8C4B21048C07E022811D10E4832
S31508004660007F002810D10D488079AA2804D10B486C
S31508004670C471012108480177AA2C05D1074884711D
S3150800468002E0204602F084FE0221024800F045F8C6
S3150800469010BD000000380140EC03002098050020FA
S315080046A010B504462146054800F09CF800BF0121D4
S315080046B0024800F03AF80028F9D010BD0038014049
S315080046C070B505460E4600247E2000F0B1FA00BFFC
S315080046D020E0042C19DD701EA04216DD285D7E2818
S315080046E006D17D20FFF7DCFF5E20FFF7D9FF0FE03C
S315080046F0285D7D2805D1FFF7D3FF5D20FFF7D0FFA2
S3150800470006E0285DFFF7CCFF02E0285DFFF7C8FF4B
S31508004710601C84B2B442DCDB70BD416170478269BB
S31508004720520852000A438261704702469068084060
S31508004730002801D0012070470020FCE70246D06817
S315080047400840002801D0012070470020FCE7002A15
S3150800475003D003690B43036102E003698B430361DA
S315080047607047000070B504460D460026E069302102
S31508004770884329790843E061E06944218843A97997
S315080047800843E061E06980088000297A0843E0610F
S31508004790A0691821884369890843A061A069042192
S315080047A08843297B0843A0610B48844203D1FFF75D
S315080047B0A7F8064602E0FFF791F80646304629684C
S315080047C0FDF7A8F80009206230462968FDF7A2F827
S315080047D00007000F606270BD003801400146486856
S315080047E0C0B27047CAB2026070474B21C901016066
S315080047F03021017100218171017218214181002146
S315080048000173704710B51C484088030000F087FA0A
S315080048100504111E292A2B0017485830008FFF213E
S315080048201B31884204DA01211348418000F020FA3E
S3150800483019E011485830008FFF210531884204DA03
S3150800484002210D48418000F013FA0CE00A4858305E
S31508004850008FF62804DA03210748418000F008FA99
S3150800486001E000E000BF00BF03487830407F002821
S3150800487001D100F0FDF910BD7403002010B53048D1
S315080048804088002806D0012813D0022820D0032803
S3150800489054D12CE080210920C006FEF78AFB0121AD
S315080048A02848FEF786FB10210920C006FEF781FB83
S315080048B044E001212348FEF77CFB80210920C0063D
S315080048C0FEF775FB10210920C006FEF770FB35E0E0
S315080048D080210920C006FEF76CFB01211948FEF766
S315080048E066FB10210920C006FEF761FB26E0164983
S315080048F04868CD21FDF70EF8C007C00F002805D17E
S3150800490080210920C006FEF752FB0DE00E494868D3
S31508004910CD21FCF7FFFFC007C00F002804D0802177
S315080049200920C006FEF745FB01210648FEF73FFBB6
S3150800493010210920C006FEF73AFB00BF00BF10BDD4
S3150800494074030020000400480C02002010B59F489C
S31508004950807E030000F0E3F90504336CAFFAF80033
S315080049609A482038008FFF211031884202DB012146
S315080049709648817640219648FEF710FB00281DD000
S3150800498094494868FF21F531FCF7C4FFC007C00FFA
S31508004990002805D180210920C006FEF708FB04E09F
S315080049A080210920C006FEF704FB10210920C00655
S315080049B0FEF7FDFA01218648FEF7F9FA03E1834876
S315080049C02038008FFF212531884202DB02217F48EB
S315080049D0817640217E48FEF7E1FA002827D07D49F6
S315080049E04868FF21F531FCF795FFC007C00F00287E
S315080049F004D101217648FEF7DAFA03E0012174486A
S31508004A00FEF7D7FA80210920C006FEF7D0FA102152
S31508004A100920C006FEF7CBFA6C487838408801288A
S31508004A2005D0012169487838418000F021F9CAE0AB
S31508004A3066482038008FFF212731884202DD03218E
S31508004A406248817640216248FEF7A8FA002831D0EC
S31508004A5060494868FF21F531FCF75CFFC007C00FC5
S31508004A6000280ED180210920C006FEF7A2FA0121EE
S31508004A705748FEF79EFA10210920C006FEF799FA54
S31508004A800DE080210920C006FEF791FA10210920C1
S31508004A90C006FEF78CFA01214D48FEF788FA4B4806
S31508004AA078384088002805D0002148487838418061
S31508004AB000F0DEF887E040214548FEF76FFA002847
S31508004AC041D0012109030920C006FEF767FA00282C
S31508004AD007D04048806D4049884202D904213B48A6
S31508004AE081763C494868FF21F531FCF713FFC0077A
S31508004AF0C00F00280ED180210920C006FEF759FAFA
S31508004B0001213348FEF755FA10210920C006FEF7A1
S31508004B1050FA0DE080210920C006FEF748FA102158
S31508004B200920C006FEF743FA01212948FEF73FFA95
S31508004B30264878384088002805D000212348783848
S31508004B40418000F095F83EE03CE0FFE74021204830
S31508004B50FEF724FA002834D01C4878384088002804
S31508004B6005D0002119487838418000F081F81948A5
S31508004B70406D1A4988420ED280210920C006FEF7E8
S31508004B8018FA01211248FEF714FA10210920C00666
S31508004B90FEF70FFA0DE080210920C006FEF707FA96
S31508004BA010210920C006FEF702FA01210848FEF77F
S31508004BB0FEF9064840300079012802D1032103484E
S31508004BC0817600E000BF00BF10BD0000EC030020A6
S31508004BD0000400480C020020941100003075000003
S31508004BE00348806840084000014988607047000013
S31508004BF0002C004080210143014A116070470000E3
S31508004C00002C004003488068002801D00120704726
S31508004C100020FCE7002C004010B5FFF7F3FF002842
S31508004C2004D0FFF7DDFF662000F002F810BD000093
S31508004C304106490E014A116070470000002C0040E9
S31508004C4004494968FF22813291430143014A516070
S31508004C5070470000002C004004494968C909C90189
S31508004C604206520E1143014A51607047002C00401B
S31508004C7010B57E20FFF7DCFF0948FEF71DF8094945
S31508004C80094801850621283000F018FA0649283116
S31508004C9088814022024904482830FEF74AF810BDA8
S31508004CA000B00008FBAA00004C03002070B50546BA
S31508004CB00C460121C802FEF7E1FDFF208130FFF70F
S31508004CC0BFFF2046FFF7C8FF2846FFF793FF70BDD2
S31508004CD00FB410B503A9044B044A029800F080F8F3
S31508004CE010BC08BC04B01847AD6E000804020020CA
S31508004CF02021020C01D010211046020A01D01046CC
S31508004D000839020901D01046091F820801D0104649
S31508004D10891E420801D0881E7047081A704730B4A9
S31508004D207446641E2578641CAB4204D3635D5B003D
S31508004D30E31830BC18471D46F8E7000010B50028F0
S31508004D4019DB1A4A03231B02D21883089B00D25880
S31508004D508307DC0EFF23A3409A438B071B0E8407A9
S31508004D60E40EA3401A43114B032424021B1984089A
S31508004D70A4001A5118E00E4A03071B0F083B9B08AC
S31508004D809B00D2588307DC0EFF23A3409A438B0768
S31508004D901B0E8407E40EA3401A43054B0407240F91
S31508004DA0083CA408A4001A5110BD000000E100E068
S31508004DB01CED00E002E008C8121F08C1002AFAD15B
S31508004DC070477047002001E001C1121F002AFBD17D
S31508004DD0704700000149086070470000080200207B
S31508004DE0FFB58FB00F460446002606E025280AD0F0
S31508004DF0129A11999047641C761C20780028F5D1E0
S31508004E00304613B0F0BD00250121A14A009500E007
S31508004E100543641C23780846203B98401042F7D186
S31508004E2020782E2815D1042005436078641C2A288A
S31508004E300AD101CF641C00900BE000990A22514365
S31508004E4030394018641C0090207801463039092909
S31508004E50F3D920786C280ED004DC4C2813D06A28A5
S31508004E6012D104E074280ED07A280DD10BE0012067
S31508004E704005054307E00121090562780D43824292
S31508004E8001D16D18641C641C2078864669284AD0AE
S31508004E9008DC0028B4D058286DD0632810D06428C0
S31508004EA008D140E070286BD0732812D0752860D0DE
S31508004EB0782860D0129A704611999047761CE5E0DA
S31508004EC03878694608720020487202A801900120C5
S31508004ED003E0386801900020C0433F1D69070CD5E0
S31508004EE0002500E06D1C00998D420FDA8542F9DB3A
S31508004EF00199495D0029F5D108E0002500E06D1CFF
S31508004F008542FCDB0199495D0029F8D1761907E04D
S31508004F10019801990078491C0191129A11999047B4
S31508004F206D1EF5D2B2E00A20029000216802400FF9
S31508004F30039102280CD001CFC117844600290DDA47
S31508004F406246084652420021814194462D2008E0D7
S31508004F50FF1DFF08FF0003CF8446EFE7280504D5A9
S31508004F602B206A46107401203CE0E8073AD020203E
S31508004F70F7E70A2000E0102000210391029007E0DD
S31508004F801020029000210420054308200391009078
S31508004F906802400F022810D001CF00218446002065
S31508004FA00D9028071FD5704670280CD0029A10203D
S31508004FB0039B42401A430CD015E0FF1DFF08FF0073
S31508004FC003CF8446EBE740206A46107401200D9013
S31508004FD00CE06046084306D030206A4610747046D6
S31508004FE0507402200D907046582804D029A00190CC
S31508004FF00DA80E900DE02CA0F9E76046039B029AD7
S31508005000FDF714F8019B84469B5C0E9A521E0E927D
S31508005010137060460843F0D10E9805A9081A203087
S315080050200190680701D5009801E0012000900199D8
S31508005030884203DD01460198081A00E00020002591
S31508005040009006E004A8129A405D119990476D1CDD
S31508005050761C0D988542F5DB04E0129A30201199EA
S315080050609047761C0099481E00900029F5DC08E058
S315080050700E980E990078491C0E91129A119990472C
S31508005080761C0199481E01900029F1DC641CB4E6DF
S315080050900928010030313233343536373839616200
S315080050A063646566000000003031323334353637C4
S315080050B038394142434445460000000010B50246CF
S315080050C00023002901D1002010BD03E01488921C9A
S315080050D0E01883B208464C1EA1B20028F6D118463D
S315080050E0F2E7000010B5C148407F002865D11021BD
S315080050F00920C006FDF75BFF80210920C006FDF7E1
S3150800510056FF0121BA48FDF752FF0020B749403142
S315080051108873002301221946184602F06FFF002300
S315080051201A461946184602F069FFB2484068FF2138
S31508005130F531884204D20421AD48FDF73AFF53E120
S315080051400421AB48FDF733FFAA484068AA498842BC
S31508005150F5D9A64820308078002817D1A548406898
S315080051607D214901884201D2FFF74CFB0821A0485E
S31508005170FDF71DFF00219D48C17700209B4940315E
S31508005180487088709B49486248630CE040219848FB
S31508005190FDF704FF002806D00021944840308173AB
S315080051A001214038417720210920C006FDF7FFFE7E
S315080051B07D2040018F49486016E18C484030807B4D
S315080051C00300FFF7ACFD060471B4FDFCFB7000207C
S315080051D0864940314870887086494862486300238A
S315080051E001221946184602F009FF00231A461946F5
S315080051F0184602F003FF7D482038418D018620308D
S31508005200C07E012808D17B4840697C49884202D97A
S3150800521000217648C17610BD764840687D2109018F
S31508005220884228D90020764908707048203080784E
S31508005230002802D16F49486002E072486D4948600B
S3150800524040216B48FDF7AAFE00280CD1FFF7DAFAD1
S3150800525008216748FDF7ABFE7E20FFF7E9FC1E2014
S31508005260FDF76AFB02E000206249486004216048B5
S31508005270FDF79DFE17E020210920C006FDF799FEDF
S3150800528008215B48FDF795FE5A484068FF21F5312D
S31508005290884208D9554878384089002803D104211E
S315080052A05348FDF784FE9EE052484068FF21F531D9
S315080052B0884204D204214E48FDF77BFE03E0042110
S315080052C04B48FDF774FE4948C07E052817D10022D1
S315080052D00121084601F0B4F844482038018D4030D1
S315080052E0C08A814205DA64220121002001F0A8F86B
S315080052F007E000220121104601F0A2F801E0FEF7BE
S315080053003BFF3A482038418D4030C08A81420DDB48
S3150800531036482038018D4030C08A814206DB00209D
S315080053203449486002203149403188735BE031488E
S315080053304068FF21F531884204D204212C48FDF744
S3150800534038FE03E004212A48FDF731FE2948406863
S315080053502D49884221D925482030C08AD2281CD117
S3150800536022482030808BCF2813DB20482030808BC2
S31508005370D5280EDA01201D49403108721D48006EF5
S315080053801E49884209D90122FE21672002F099FDAB
S3150800539003E000201549403108721448C07E0528EC
S315080053A01BD100220121084601F04AF80F4820388F
S315080053B0018D4030C08A814209DA02E012E010E02D
S315080053C00EE03C220121002001F03AF807E0002215
S315080053D00121104601F034F801E0FEF7CDFE02E0A7
S315080053E001E000E000BF00BF00BF14E7EC030020A7
S315080053F0000400480C020020B80B000088130000C7
S31508005400C4000020C40900001027000010B5C048D9
S31508005410407F002865D110210920C006FDF7C7FD89
S3150800542080210920C006FDF7C2FD0121B948FDF714
S31508005430BEFD0020B6494031887300230122194673
S31508005440184602F0DBFD00231A461946184602F0F4
S31508005450D5FDB1484068FF21F531884204D20421C0
S31508005460AC48FDF7A6FD50E10421AA48FDF79FFDCB
S31508005470A9484068A9498842F5D9A54820308078C6
S31508005480002817D1A44840687D214901884201D2E5
S31508005490FFF7B8F908219F48FDF789FD00219C48C8
S315080054A0C17700209A494031487088709A49486205
S315080054B048630CE040219748FDF770FD002806D0A8
S315080054C00020934940318873012191484177202172
S315080054D00920C006FDF76BFD7D2040018E49486016
S315080054E013E18B484030807B0300FFF718FC060465
S315080054F075B1FDFCFB7400208549403148700021D8
S3150800550083484030817000208349486248630023FD
S3150800551001221946184602F071FD00231A4619465B
S31508005520184602F06BFD7A482038418D01862030F6
S31508005530C07E012808D1784840697949884202D94D
S3150800554000217348C17610BD734840687D21090162
S31508005550884228D90020734908706D482030807821
S31508005560002802D16C49486002E06F486A494860E1
S3150800557040216848FDF712FD00280CD1FFF742F9D3
S3150800558008216448FDF713FD7E20FFF751FB1E2016
S31508005590FDF7D2F902E000205F49486004215D4822
S315080055A0FDF705FD17E020210920C006FDF701FDDE
S315080055B008215848FDF7FDFC57484068FF21F5319A
S315080055C0884208D9524878384089002803D10421EE
S315080055D05048FDF7ECFC97E04F484068FF21F5314D
S315080055E0884204D204214B48FDF7E3FC03E004217A
S315080055F04848FDF7DCFC4648C07E062817D100223D
S315080056000121104600F01CFF41482038418D4030EA
S31508005610C08A814205DA50220121084600F010FFAF
S3150800562007E000220121084600F00AFF01E003F026
S3150800563091FB37482038418D4030C08A814206DBCD
S3150800564000203549486002203149403188735BE0C3
S3150800565031484068FF21F531884204D204212D489B
S31508005660FDF7A7FC03E004212A48FDF7A0FC2A4819
S3150800567040682E49884221D925482030C08AD22838
S315080056801CD123482030808BCF2813DB20482030BC
S31508005690808BD5280EDA01201D49403108721E4834
S315080056A0006E1F49884209D90122FE21672002F0AF
S315080056B008FC03E000201649403108721448C07EF1
S315080056C006281BD100220121104600F0B9FE104819
S315080056D02038418D4030C08A814209DA3C220121B6
S315080056E0084602E00FE00DE00BE000F0A9FE07E037
S315080056F000220121084600F0A3FE01E003F02AFB80
S3150800570002E001E000E000BF00BF00BF1BE70000A9
S31508005710EC030020000400480C020020B80B00002F
S3150800572088130000C4000020C409000010270000E8
S3150800573010B56E48407F002865D110210920C006A3
S31508005740FDF735FC80210920C006FDF730FC012154
S315080057506748FDF72CFC002164484030817300231C
S3150800576001221946184602F049FC00231A46194632
S31508005770184602F043FC5F484068FF21F53188422D
S3150800578004D204215A48FDF714FCADE00421584818
S31508005790FDF70DFC5748406857498842F5D95348E4
S315080057A020308078002817D1524840687D21490169
S315080057B0884201D2FFF726F808214D48FDF7F7FB86
S315080057C000214A48C177002048494031487088700E
S315080057D04849486248630CE040214548FDF7DEFB2E
S315080057E0002806D000214148403081730121403805
S315080057F0417720210920C006FDF7D9FB7D2040010D
S315080058003C49486070E039484030807B002804D025
S31508005810012866D0022866D164E00021334840306A
S3150800582041700020314940318870324948624863E6
S315080058302E482038418D01862030C07E012808D1A7
S315080058402C4840692D49884202D900212748C1764B
S3150800585010BD284840687D210901884228D90020C2
S3150800586027490870214820308078002802D121492C
S31508005870486002E023481F49486040211C48FDF75C
S315080058808DFB00280CD1FEF7BDFF08211848FDF74F
S315080058908EFB7E20FFF7CCF91E20FDF74DF802E0BF
S315080058A000201449486004211148FDF780FB17E0E1
S315080058B020210920C006FDF77CFB08210C48FDF7CE
S315080058C078FB0C484068FF21F531884208D907481B
S315080058D078384089002803D104210548FDF767FB7D
S315080058E001E000E000BF00BF00BFB1E7EC03002005
S315080058F0000400480C020020B80B000088130000C2
S31508005900C4000020C4090000F0B587B00020069046
S31508005910059000240025049000260027FA48807A7E
S31508005920012815D1F94840697D21090188420FD916
S315080059300021F54881720020F4494861F44908803D
S31508005940F4490870FF210131F148801DFCF725F85C
S31508005950ED484038007F012879D17E20FFF768F9A5
S31508005960EB48C0790002EA49097A08430690E848F4
S31508005970407A0590E648847AC67A0246117B507BBF
S3150800598001F05AFE0746E24AD17A107B01F054FE2E
S3150800599005460021DC4840380177012140308172F4
S315080059A00020DA494861DC4A0698811A90426FD08D
S315080059B02EDCDA4A811A90426BD016DCD84A811A54
S315080059C0904267D00ADC442834D0D64940180028CB
S315080059D07BD001287AD0022879D142E2012977D0F2
S315080059E0022976D00329F7D190E2302972D008DC53
S315080059F00D2970D00E296FD00F296ED01F29EBD133
S31508005A0069E331296AD0382969D04129E4D1CEE33E
S31508005A10084634380300FFF782F917F2F1F0EFF37E
S31508005A20EDEC5A5A5A5AC1D9EBEA5A5A222E88A28A
S31508005A304B705A00059806280AD1BB4800780028FA
S31508005A400CD102F07BFA0120B749087006E0EFE3B3
S31508005A500598152802D1012002F070FAEAE3AA484F
S31508005A60807B002806D0A8486038028D418D00202A
S31508005A7002F084F9DEE3002C0DD1A3486038408D8E
S31508005A8000231A46F0210090FE2002F0E6F90EE007
S31508005A90BFE361E2FDE1012C09D19B486038008D26
S31508005AA001230022F0210090FE2002F0D6F9C1E37E
S31508005AB0002C15D195486830408800231A46F321F2
S31508005AC00090FE2002F0C9F916E0A7E1B5E1B0E3BF
S31508005AD0FDE107E215E360E2AAE2F4E235E349E311
S31508005AE0012C09D189486830808901230022F321D5
S31508005AF00090FE2002F0B1F99CE3002C03D1834804
S31508005B006830458002E08148683085817F48683082
S31508005B108089FF21F531884206DA01F0A5F90022CD
S31508005B20FE21F42002F0CDF984E3002C0AD177484F
S31508005B306830808800231A46F1210090FE2002F082
S31508005B408CF90BE0012C09D170486830C089012313
S31508005B500022F1210090FE2002F07FF96AE3002C72
S31508005B6003D16A486830858004E0012C02D1674871
S31508005B706830C581654868308088FF21F5318842DC
S31508005B800BDC62486830C089884206DC01F06CF993
S31508005B900022FE21F22002F094F94BE3002C0AD1F0
S31508005BA05A486830C08800231A46E9210090FE202A
S31508005BB002F053F909E0012C07D11920012300222C
S31508005BC0E9210090FE2002F048F933E3002C02D1C7
S31508005BD04E486830C580FF202D30854206DA01F030
S31508005BE043F90022FE21EA2002F06BF922E352E093
S31508005BF031E06DE016E003E0D0E0F5E0AEE0C2E0AB
S31508005C00002C0DD14148683000896421484380B290
S31508005C1000231A46E2210090FE2002F01EF900E059
S31508005C2000BF07E3002C07D164212846FBF788FE4E
S31508005C3081B2364868300181344868300089FF21CE
S31508005C40F531884206DC01F00FF90022FE21E32037
S31508005C5002F037F9EEE2002C0DD12C486830408965
S31508005C606421484380B200231A46EB210090FE20A7
S31508005C7002F0F3F80EE0012C0CD124486830008AB3
S31508005C806421484380B201230022EB210090FE20C4
S31508005C9002F0E3F8CEE2002C08D164212846FBF78F
S31508005CA04FFE81B219486830418109E0012C07D1BD
S31508005CB064212846FBF744FE81B214486830018205
S31508005CC001F0D2F80022FE21EC2002F0FAF8B1E247
S31508005CD0012C2BD10C48B838408803280ADA0A4820
S31508005CE0B8384089002805D101210748817300206A
S31508005CF0064948600022FE21E42002F0E2F801216C
S31508005D0001484038417728E02C0400200C02002086
S31508005D1098050020F1010020AAFE000058FE0000A8
S31508005D2054FE0000AF01FFFF00020020002C0FD137
S31508005D300021FE484177403081730022FE21E4208D
S31508005D4002F0BFF80020FA490870FA49486004E0F2
S31508005D500022FE21E42002F0B4F86BE2002C10D1F8
S31508005D60F548C07A32280DDCF348C17AF148683024
S31508005D70418201F079F80022FE21DF2002F0A1F825
S31508005D8000E000BF56E2EB486830408A00231A4616
S31508005D90DE210090FE2002F060F84BE2002C10D1C4
S31508005DA0E548C07A32281EDCE348C17AE148683003
S31508005DB0818201F059F80022FE21E12002F081F8E3
S31508005DC011E0012C0FD1DC48C07A32280BDCDA4806
S31508005DD0C17AD8486830C18201F046F80022FE210F
S31508005DE0E12002F06EF825E2002C0AD1D14868308D
S31508005DF0808A00231A46E0210090FE2002F02DF842
S31508005E000BE0012C09D1CB486830C08A0123002257
S31508005E10E0210090FE2002F020F80BE2C749C548B1
S31508005E2068308183C1830184418401F01DF8002212
S31508005E30FE21512002F045F8FCE1002C10D1002E7D
S31508005E4003D1BA48203007830AE0012E03D1B748A8
S31508005E502030478304E0022E02D1B44820308783DD
S31508005E60E8E1002C14D1FDF751FB04900498000CCE
S31508005E7000231A4653210090FE2001F0EEFF0498F5
S31508005E8080B20123002253210090FE2001F0E5FF95
S31508005E90D0E1002C0CD1A7486830C08B0090A548EB
S31508005EA06830838B00225421FE2001F09CFF0DE010
S31508005EB0012C0BD19F486830408C00909D48683073
S31508005EC0038C01225421FE2001F08DFFB2E1002C43
S31508005ED007D101219548C176002202219848FEF78C
S31508005EE036FCA7E1002C10D1FF2101319248801D14
S31508005EF0FBF753FD00209049088002218B48C176A4
S31508005F000022FE21562001F0DCFF93E1002C16D179
S31508005F10002186484030C171002087490880032146
S31508005F208248C1760121417740308173002081493A
S31508005F3048600022FE21572001F0C3FF0BE0012C28
S31508005F4009D100217948C176403081730122FE21AA
S31508005F50572001F0B6FF6DE1002C16D100217348D9
S31508005F604030C17100207449088004216F48C17609
S31508005F70012141774030817300206E494860002234
S31508005F80FE21582001F09DFF06E0012C04D10021D6
S31508005F906648C176403081734CE1002C16D100204A
S31508005FA06549088006216148C1760121417740305C
S31508005FB0817300205F494860B4215C482030C18263
S31508005FC00022FE21652001F07CFF30E0012C16D16D
S31508005FD000205949088006215448C1760121417795
S31508005FE040308173002053494860D2214F48203001
S31508005FF0C1820022FE21652001F063FF17E0022C12
S3150800600015D100204C49088006214848C17601214F
S31508006010417740308173002046494860F021434863
S315080060202030C1820022FE21652001F04AFF01E1ED
S31508006030002C16D100204049088005213B48C1762E
S31508006040012141774030817300203A494860B421E4
S3150800605036482030C1820022FE21662001F031FF39
S3150800606030E0012C16D100203349088005212F483D
S31508006070C176012141774030817300202D4948605F
S31508006080D2212A482030C1820022FE21662001F052
S3150800609018FF17E0022C15D1002027490880052192
S315080060A02248C17601214177403081730020214979
S315080060B04860F0211D482030C1820022FE2166205A
S315080060C001F0FFFEB6E000211848C1760020174906
S315080060D040318873AEE0002C08D107211348C176F9
S315080060E00022FE21772001F0ECFE09E0012C07D101
S315080060F000210E48C1760122FE21772001F0E1FE3B
S3150800610098E0002C20D164220121002000F098F9A3
S3150800611000220121084600F093F901210348403086
S3150800612081730022FE2188200CE00000EC03002089
S31508006130000200200C020020980500200410000030
S315080061400038014001F0BDFE74E0002C11D1642234
S315080061500121084600F074F900220121104600F0DA
S315080061606FF90121354881730022FE21892001F04B
S31508006170A8FE5FE0324933480068FBF772FC0190DD
S31508006180FBF7C9FE80B22E4903902F480068FBF73B
S3150800619068FC0190FBF7BFFE80B20290039800905E
S315080061A000229021FE20029B01F01DFE42E0002CF9
S315080061B02ED1002E09D12548C7830022FE21522060
S315080061C001F07FFE00F050FE22E0012E09D11F48A3
S315080061D0878300F049FE0122FE21522001F071FE5C
S315080061E016E0022E09D11948478400F03DFE022226
S315080061F0FE21522001F065FE0AE0032E08D113485D
S31508006200078400F031FE0322FE21522001F059FED8
S3150800621010E0002C0BD101210848817340384177E2
S3150800622001200649C872002008496839486001E01B
S3150800623001E000BF00BF07B0F0BD00002C0400203D
S3150800624000007A44900100208C010020740200208E
S31508006250F0B589B000200890079006904048007F66
S3150800626001287BD13F488079AA2874D13D48C07956
S3150800627032286DDA3B48C079002869DD3949C97981
S3150800628008461938FBF7FAFD08900898FBF776FEDA
S315080062900446354A354BFBF711FD0022344B019174
S315080062A00090FBF759FC0391029032480068FBF70F
S315080062B065FE0646039B029AFBF768FD0591049066
S315080062C0FBF784FE07902C490798FBF7CAFB0446A0
S315080062D0FBF721FE81B2294841830898FBF74EFE59
S315080062E00646214A214BFBF7E9FC04460022204BCF
S315080062F0FBF732FC0391029021480068FBF73EFE4B
S3150800630001910090039B029AFBF740FD05910490CA
S31508006310FBF75CFE069018490698FBF7A2FB0446B5
S31508006320FBF7F9FD81B215480183408B00901348AD
S31508006330038B00226021FE2001F055FD0122FE217B
S31508006340562001F0BEFD00F08FFD00210448C176FD
S3150800635000210348C17600210148017709B0F0BD44
S31508006360EC03002098050020091B9E5E29CB703F90
S315080063700000F03F8C01002000007A4474020020DF
S31508006380900100202A494A88498A511A814209DB24
S31508006390274968398968264A683AD1620021254A18
S315080063A011701BE022494988814217DC2149097886
S315080063B0002913D120490A8F40310A8201211D4A3A
S315080063C011701B4968398968194A683AD26A891A64
S315080063D0174A683A516211468968516314498A888E
S315080063E0898A511A814209DB0021144A1170104921
S315080063F0683989680E4A683A116318E00C49898831
S31508006400814214DC0D490978002910D10A490A8FFE
S3150800641040314A820121094A11700549683989685B
S31508006420034A683A126B891A014A683A91627047B8
S3150800643074020020E4000020CC030020E5000020C0
S3150800644070B505460E461446002E02D0012E4AD1D6
S3150800645020E0002D02D0012D1AD10CE06021012088
S315080064608007FDF7B3FD002101208007FDF732FE06
S315080064701E4804700CE0602101208007FDF7AEFD80
S31508006480002101208007FDF72EFE1948047000BF81
S3150800649000BF28E0002D02D0012D22D110E01348BC
S315080064A00078A0420BD0602101208007FDF78EFD01
S315080064B0214601208007FDF70DFE0C48047010E008
S315080064C00B480078A0420BD0602101208007FDF719
S315080064D085FD214601208007FDF705FE0448047066
S315080064E000BF00BF00BF00BF70BD0000A3010020B1
S315080064F0A401002010B5F348407F012879D1F1485E
S315080065004030407B0028F9D1EE48C07F0300FEF7F3
S3150800651006FC0805075DB0FDFCFBFAF9002010BD76
S31508006520E9494868FF219131FBF7F4F98007800FA4
S31508006530002809D180210920C006FCF738FD012171
S31508006540E248FCF734FD3AE0DF494868FF2191311B
S31508006550FBF7E0F98007800F012809D1802109207F
S31508006560C006FCF726FD0121D848FCF720FD26E0E9
S31508006570D5494868FF219131FBF7CCF98007800F90
S31508006580022809D180210920C006FCF710FD012147
S31508006590CE48FCF70CFD12E0CB494868FF21913143
S315080065A0FBF7B8F98007800F032808D10121C748EF
S315080065B0FCF7FFFC80210920C006FCF7F8FC102137
S315080065C00920C006FCF7F3FC0120A8E7BE49486885
S315080065D0C821FBF79FF98007800F00280AD1802180
S315080065E00920C006FCF7E3FC0121B848FCF7DFFCEC
S315080065F038E065E1B4494868C821FBF78BF980079C
S31508006600800F012809D180210920C006FCF7D1FC9A
S315080066100121AE48FCF7CBFC24E0AB494868C82109
S31508006620FBF778F98007800F022809D18021092015
S31508006630C006FCF7BCFC0121A448FCF7B8FC11E035
S31508006640A1494868C821FBF765F98007800F032828
S3150800665008D101219D48FCF7ACFC80210920C00621
S31508006660FCF7A5FC10210920C006FCF7A0FC0120B8
S3150800667055E795494868C821FBF74CF98007800F0C
S31508006680002809D180210920C006FCF790FC0121C9
S315080066908E48FCF78CFC3DE08B494868C821FBF71F
S315080066A039F98007800F012809D180210920C00601
S315080066B0FCF77FFC01218548FCF779FC2AE0824932
S315080066C04868C821FBF726F98007800F022809D1F8
S315080066D080210920C006FCF76AFC01217B48FCF7EB
S315080066E066FC17E078494868C821FBF713F9800764
S315080066F0800F03280ED101217448FCF75AFC80212B
S31508006700092004E0DBE0B2E05FE034E009E0C0061F
S31508006710FCF74DFC10210920C006FCF748FC0120B7
S31508006720FDE669494868FF212D31FBF7F3F8C007F4
S31508006730C00F002805D180210920C006FCF737FCC8
S315080067400EE061494868FF212D31FBF7E3F8C007E1
S31508006750C00F002804D080210920C006FCF729FCB8
S3150800676010210920C006FCF722FC01215748FCF736
S315080067701EFC0120D3E654494868FF219131FBF7F6
S31508006780C9F8C007C00F002805D180210920C00616
S31508006790FCF70DFC0EE04C494868FF219131FBF7E8
S315080067A0B9F8C007C00F002804D080210920C00608
S315080067B0FCF7FFFB10210920C006FCF7F8FB0121B6
S315080067C04248FCF7F4FB0120A9E63F494868C8217E
S315080067D0FBF7A0F88007800F002809D1802109203F
S315080067E0C006FCF7E4FB01213848FCF7E0FB37E07C
S315080067F035494868C821FBF78DF88007800F0128BE
S3150800680009D180210920C006FCF7D3FB01212F48B6
S31508006810FCF7CDFB24E02C494868C821FBF77AF839
S315080068208007800F022809D180210920C006FCF7BD
S31508006830BEFB01212548FCF7BAFB11E0224948684E
S31508006840C821FBF767F88007800F032808D10121C4
S315080068501E48FCF7AEFB80210920C006FCF7A7FB03
S3150800686010210920C006FCF7A2FB012057E61649AD
S315080068704868C821FBF74EF8C007C00F002805D1A5
S3150800688080210920C006FCF792FB0DE00E494868F6
S31508006890C821FBF73FF8C007C00F002804D08021A5
S315080068A00920C006FCF785FB10210920C006FCF765
S315080068B07EFB01210548FCF77AFB01202FE600BF85
S315080068C000BF2CE6EC0300200C0200200004004860
S315080068D010B5FE48807B002871D0FC486038408D92
S315080068E0FF217D31884204DCF8486038008D8842F3
S315080068F01CDDF6484038C07F002817D1F448408888
S315080069000A2813DDF2484088F24988420EDAF04830
S3150800691080880A280ADDEE488088884206DA002040
S31508006920ED4948600321E9484038C177EA48006CD8
S31508006930EA4988420AD9E5484038C07F002805D187
S31508006940E54948600321E1484038C177DF48807B44
S31508006950042835D1DD484078002828D1DB4820387E
S31508006960C07801281ED1DC48006DDD4988422ED941
S315080069700020D9490865D5486038C18D008D814207
S315080069800BDBD2484038C07F002820D1D249486066
S315080069900721CE484038C17719E0CC486038018DC8
S315080069A0C18514E0C9486038018DC1850FE0002013
S315080069B0C9490865C5486038018DC18507E028E0E2
S315080069C00020C5490865C1486038018DC185BF48A2
S315080069D0807B012828D1BD482038007901281ED19E
S315080069E0BD48C06CBE49884225D90020BA49C8644A
S315080069F0B6486038818D408D81420BDBB3484038FC
S31508006A00C07F002817D1B44948600721AF484038ED
S31508006A10C17710E0AD486038418D81850BE0AB4801
S31508006A206038418D818506E00020AB49C864A748D7
S31508006A306038418D8185A5484038407F012877D147
S31508006A40A2484038C07F00280BD0002301221946EF
S31508006A50184601F0D3FA00231A461946184601F0DB
S31508006A60CDFA9A484038C07F0300FEF758F9080562
S31508006A70073C71A4D7FDFCFB002010BD9648406872
S31508006A80E121C900884229D910210920C006FCF74E
S31508006A908EFA80210920C006FCF789FA012191485F
S31508006AA0FCF785FA0120894948730846C07A002808
S31508006AB007D1894948600021844840384177C17721
S31508006AC008E085484068AF210901884202D90020BC
S31508006AD08149486001207D49087302E000207B490E
S31508006AE048730120C9E77C4840687F4988422AD90B
S31508006AF010210920C006FCF75AFA80210920C00691
S31508006B00FCF755FA01217748FCF751FA01206F493D
S31508006B1048730846C07A00280BD16F49486000219F
S31508006B206A4840384177C17700206B4948600DE0D4
S31508006B3029E169484068AF210901884206D9002041
S31508006B406549486002E0002060494873012094E7DF
S31508006B50614840686549884228D910210920C0063D
S31508006B60FCF725FA80210920C006FCF720FA012146
S31508006B705C48FCF71CFA0120544948730846C07A59
S31508006B8000280AD1544948600021504840384177C6
S31508006B90C1770020504948600BE04F484068544987
S31508006BA0884206D900204C49486002E0002147483F
S31508006BB04173012061E7484840687D210901884200
S31508006BC027D910210920C006FCF7F1F980210920F0
S31508006BD0C006FCF7ECF901214248FCF7E8F9012167
S31508006BE03A484173C07A00280AD13B4948600021D7
S31508006BF0364840384177C1770020374948600BE06E
S31508006C00354840683649884206D9002032494860E6
S31508006C1002E000202D49487301202EE72E484068DF
S31508006C20E121C90088422CD910210920C006FCF7A9
S31508006C30BEF980210920C006FCF7B9F901212948C7
S31508006C40FCF7B5F9012121484173C07A00280ED115
S31508006C502149486000211D4840384177C177002006
S31508006C601D4902E08EE05AE010E048600CE01A4840
S31508006C704068AF210901884206D9002016494860B4
S31508006C8002E00021114841730120F6E612484068E7
S31508006C901749C83988423DD910210920C006FCF792
S31508006CA086F980210920C006FCF781F901210D48E3
S31508006CB0FCF77DF90120054948730846C07A002883
S31508006CC01FD1054948600021004813E02C04002024
S31508006CD074010020E60F00000C020020701101006C
S31508006CE0B80B000000040048A4060000C409000010
S31508006CF0AC0D000040384177C17700202349486031
S31508006D000BE0224840682249884206D900201F49DC
S31508006D10486002E000201F4948730120ADE61B4881
S31508006D2040681D49884228D910210920C006FCF769
S31508006D303EF980210920C006FCF739F901211748D8
S31508006D40FCF735F90120134948730846C07A00282C
S31508006D500AD10E49486000210E4840384177C1776C
S31508006D6000200A4948600BE0084840680C498842F8
S31508006D7006D900200549486002E00021054841730C
S31508006D8001207AE600BF00BF77E600000C0200206B
S31508006D90CC1000002C040020A406000000040048C3
S31508006DA08C0A000010B5052421E080212C48FAF74A
S31508006DB0F4FD80212A48FBF7A9FE12212848FEF790
S31508006DC07DF92749898C88420CD125482838008DB9
S31508006DD02449884204D000F0E9FC00F045F800E0B8
S31508006DE010BD04E0002000E0401C8028FCDB2046A3
S31508006DF0611ECCB20028D8D100BF052423E080212B
S31508006E001748FAF7CAFD80211548FBF79DFE12219F
S31508006E101348FEF753F91249898C88420ED1104857
S31508006E202838008D0F49884204D000F0BFFC00F0D6
S31508006E301BF802E000F018F8D2E704E0002000E0B2
S31508006E40401C8028FCDB2046611ECCB20028D6D127
S31508006E5000BF00F0ABFC00F007F800BFC0E7000079
S31508006E6074020020FBAA000010B57E20FDF7E0FEA4
S31508006E70FBF70CFF0B490C48018512212830FEF759
S31508006E801DF9094928318884802107482830FBF7ED
S31508006E9097FE7E20FDF7CCFE802103482830FBF7BD
S31508006EA09BFE10BDFBAA00004C02002070B50446EC
S31508006EB00D46E1B20548FDF795FC00BF01210348E0
S31508006EC0FDF733FC0028F9D0204670BD0038014094
S31508006ED0F0B587B000240020069005904049088B3D
S31508006EE0FAF7D7FF07463F49FAF7F8FD05463C4942
S31508006EF0088BFAF7CEFF3B490490FAF7EFFD0746F1
S31508006F00394801683846FAF7A8FD06462946FAF7C9
S31508006F10E5FD06903549888BFAF7BBFF06463449E6
S31508006F20FAF797FD054629460698FAF7D7FD05901C
S31508006F3030490598FAF795FD0546FAF7ECFF81B250
S31508006F402748C183C08B00902548838B0022542193
S31508006F50FE2000F048FF2249088BFAF79AFF2049DD
S31508006F600190C88BFAF795FF22490090FAF7B6FD0B
S31508006F7007460199FAF775FD06461A49FAF7AEFD6E
S31508006F8017490390088BFAF784FF07461549FAF75D
S31508006F90A5FD0646144801683046FAF75EFD0290DC
S31508006FA00399FAF79BFD05461149FAF701FD049086
S31508006FB0FAF7B1FF84B20A48C08B0F49884204DB4E
S31508006FC00748C08B0D49884204DD0222FE2157205E
S31508006FD000F077FF054840384485204607B0F0BDE5
S31508006FE07402002000007A44900100200C0400205E
S31508006FF00000C84100247449B80B0000881300003B
S31508007000F0B587B000240020069005904049488BCB
S31508007010FAF73FFF07463F49FAF760FD05463C4940
S31508007020488BFAF736FF3B490490FAF757FD0746AF
S31508007030394801683846FAF710FD06462946FAF730
S315080070404DFD06903549088BFAF723FF0646344965
S31508007050FAF7FFFC054629460698FAF73FFD05901C
S3150800706030490598FAF7FDFC0546FAF754FF81B250
S3150800707027488183C08B00902548838B00225421A2
S31508007080FE2000F0B0FE2249488BFAF702FF20499D
S315080070900190C88BFAF7FDFE22490090FAF71EFD0B
S315080070A007460199FAF7DDFC06461A49FAF716FD6E
S315080070B017490390488BFAF7ECFE07461549FAF785
S315080070C00DFD0646144801683046FAF7C6FC0290DC
S315080070D00399FAF703FD05461149FAF769FC049086
S315080070E0FAF719FF84B20D48403804850848808BA2
S315080070F00D49884204DB0648808B0C49884204DD2A
S315080071000222FE21572000F0DCFE204607B0F0BD23
S315080071107402002000007A448C0100200C04002030
S315080071200000C84100247449B80B00008813000009
S31508007130F0B587B000240020069005904049088BDA
S31508007140FAF7A7FE07463F49FAF7C8FC05463C4941
S31508007150088BFAF79EFE3B490490FAF7BFFC0746F0
S31508007160394801683846FAF778FC06462946FAF798
S31508007170B5FC06903549888BFAF78BFE06463449E6
S31508007180FAF767FC054629460698FAF7A7FC05901C
S3150800719030490598FAF765FC0546FAF7BCFE81B250
S315080071A027484184408C00902548038C01225421AD
S315080071B0FE2000F018FE2249088BFAF76AFE2049DD
S315080071C00190488CFAF765FE22490090FAF786FC8A
S315080071D007460199FAF745FC06461A49FAF77EFC6E
S315080071E017490390088BFAF754FE07461549FAF72C
S315080071F075FC0646144801683046FAF72EFC0290DC
S315080072000399FAF76BFC05461149FAF7D1FB049086
S31508007210FAF781FE84B20A48408C0F49884204DB9B
S315080072200748408C0D49884204DD0222FE2157207A
S3150800723000F047FE054840384485204607B0F0BDB3
S315080072407402002000007A44900100200C040020FB
S315080072500000C84100247449B80B000088130000D8
S31508007260F0B587B000240020069005904049488B69
S31508007270FAF70FFE07463F49FAF730FC05463C4940
S31508007280488BFAF706FE3B490490FAF727FC0746AF
S31508007290394801683846FAF7E0FB06462946FAF700
S315080072A01DFC06903549088BFAF7F3FD0646344966
S315080072B0FAF7CFFB054629460698FAF70FFC05901C
S315080072C030490598FAF7CDFB0546FAF724FE81B250
S315080072D027480184408C00902548038C01225421BC
S315080072E0FE2000F080FD2249488BFAF7D2FD20499E
S315080072F00190088CFAF7CDFD22490090FAF7EEFBCB
S3150800730007460199FAF7ADFB06461A49FAF7E6FB6E
S3150800731017490390488BFAF7BCFD07461549FAF753
S31508007320DDFB0646144801683046FAF796FB0290DC
S315080073300399FAF7D3FB05461149FAF739FB049086
S31508007340FAF7E9FD84B20A48008C0F49884204DB43
S315080073500748008C0D49884204DD0222FE21572089
S3150800736000F0AFFD054840380485204607B0F0BD5B
S315080073707402002000007A448C0100200C040020CE
S315080073800000C84100247449B80B000088130000A7
S3150800739070B5044600257E20FDF74AFCA348008800
S315080073A07D280ADD0020A1490880A1490870FF212F
S315080073B001319E48801DFAF7F0FA9D4800780300CF
S315080073C0FDF7ADFC080521364760DAF1F0EF00203D
S315080073D0964948717E2C0FD108800120944908707F
S315080073E0924801880088401C904A1080901D445499
S315080073F000201146C87002E000208C490880002051
S315080074008A4908710FE1FE2C01D0002C0FD187485C
S3150800741001880088401C854A1080901D445402202B
S315080074208349087010460079001911460871FAE078
S315080074307E4801880088401C7C4A1080901D445470
S3150800744003207B4908701046007900191146087117
S31508007450E9E0764801880088401C744A1080901D2F
S3150800746044540420724908701046007900191146E0
S3150800747008710846C470C078002802D105206C49F6
S315080074800870D0E069484079012856D15E2C1CD195
S31508007490664800797E30654908717E21634802880E
S315080074A00088401C614B1880981D8154801FC07845
S315080074B0401EC0B21946C870002802DC05205C4987
S315080074C0087000205949487155E05D2C1CD1574871
S315080074D000797D30554908717D2154480288008815
S315080074E0401C524B1880981D8154801FC078401E3E
S315080074F0C0B21946C870002802DC05204C4908703D
S3150800750000204A49487136E0484800790019474939
S315080075100871084601880088401C444A1080901D5E
S315080075204454801FC078401EC0B21146C870002857
S3150800753021DC05203E4908701DE07D2C03D1012081
S315080075403A49487117E039480079001937490871EE
S31508007550084601880088401C344A1080901D44540F
S31508007560801FC078401EC0B21146C870002802DCD1
S3150800757005202F49087056E02C480079C043401C66
S31508007580C5B27D2D05D15D2C17D106202849087076
S3150800759013E07E2D08D15E2C0FD1062024490870F1
S315080075A00BE03FE02FE011E0A54203D10620204979
S315080075B0087002E007201E4908701C4801880088E8
S315080075C0401C1A4A1080901D44542CE01748018824
S315080075D00088401C154A1080901D44547E2C08D102
S315080075E001211448017700201146088010490870C7
S315080075F008E000200D49088000210E480177002088
S315080076000B4908700FE000200949087007480188EF
S315080076100088401C054A1080901D445400201146DD
S31508007620088000E000BF00BF70BD0000980500207C
S31508007630F1010020EC03002070B502460020134635
S315080076400C461D02FF26360235402543284670BDE6
S3150800765086B004460D4626686768A0680590E06807
S3150800766004902069039060690290A0690190E0691E
S31508007670009017A0FDF72CFB31461BA0FDF728FB51
S3150800768039461CA0FDF724FB1DA00599FDF720FB34
S315080076901EA00499FDF71CFB1FA00399FDF718FB14
S315080076A020A00299FDF714FB23A00199FDF710FB12
S315080076B026A00099FDF70CFB2948416A29A0FDF789
S315080076C007FB29462BA0FDF703FB00BFFEE70000DA
S315080076D05B48617264206661756C742068616E64CB
S315080076E06C65725D0D0A00005230203D2025780D2C
S315080076F00A0000005231203D2025780D0A000000BE
S315080077005232203D2025780D0A0000005233203DD4
S315080077102025780D0A000000523132203D202578B8
S315080077200D0A0000537461636B6564204C52203D5A
S315080077302025780D0A000000537461636B65642088
S315080077405043203D2025780D0A00000053746163DC
S315080077506B656420505352203D2025780D0A0000A1
S3150800776000ED00E05343425F53484353523D2578AA
S315080077700D0A000043757272656E74204C52203DE6
S315080077802025780D0A0000000649074801850021D2
S31508007790283041805F218180C1800181002141819B
S315080077A070470000FBAA00004C03002000B51649EC
S315080077B016480185FF210531283041800A210181BB
S315080077C0A021C180CD2181801E214181AF21C181A7
S315080077D08C210182BE2181810D4901830C492539FD
S315080077E04183052141820A2181820F21C1820949EB
S315080077F08183C183018441841221FDF75FFC03491B
S315080078002831888400BD0000FBAA00004C02002035
S31508007810782100000410000010B57E20FDF708FA54
S31508007820FEF768FE012800D110BD4F48407F0128A9
S3150800783072D14D484030807B002802D001283ED1C5
S3150800784015E040214948FBF7A9FB00280CD1484818
S31508007850406D4849884209D243487838408900280B
S3150800786004D1FDF70BF801E0FDF770F878E0404920
S315080078704868FF21F531FAF74DF8C007C00F002810
S315080078800ED180210920C006FBF793FB012137485A
S31508007890FBF78FFB10210920C006FBF78AFB0DE0DA
S315080078A080210920C006FBF782FB10210920C006AB
S315080078B0FBF77DFB01212D48FBF779FB50E02A48B1
S315080078C04030807B052828D129494868FF21F531B1
S315080078D0FAF720F8C007C00F00280ED1802109202A
S315080078E0C006FBF766FB01212048FBF762FB102167
S315080078F00920C006FBF75DFB31E080210920C006A0
S31508007900FBF755FB10210920C006FBF750FB0121A8
S315080079101648FBF74CFB22E023E013484030807BF7
S3150800792006280ED180210920C006FBF740FB10214E
S315080079300920C006FBF73BFB01210C48FBF737FB88
S315080079400DE080210920C006FBF733FB012107481B
S31508007950FBF72FFB10210920C006FBF72AFB00BF07
S3150800796000BF00BF60E70000EC03002000040048E9
S315080079700C02002030750000FCF752FAFBF7DEFD1A
S31508007980FBF7FEFEFBF71AF8FAF7B2FD0B20FAF73B
S31508007990E1FC0C20FAF7DEFC0920FAF7DBFC0320F1
S315080079A0FAF7D8FC01219348FAF748FE4B20000263
S315080079B0FAF76AFF0121904841770021C177002034
S315080079C08D4940310873C87201218B482030817077
S315080079D0FBF7E8FDFCF75AFA88496320FCF784FAB6
S315080079E0FFF7E0F9FCF704FE00F0A2F982487838C0
S315080079F04089002801D1FCF741FF7F217E20FDF751
S31508007A0055F900217C48C17600207B494031087130
S31508007A10EFE07948C07E0300FDF781F90805134DAC
S31508007A208B9EB1C4D7EAFAF731FEFFF7F5FEFDF7EC
S31508007A306BFFFBF7B7FD01F0FFFA7E20FDF7F8F8BC
S31508007A40D6E0002301221946184600F0D7FA00238B
S31508007A501A461946184600F0D1FA69484068694935
S31508007A60884204D908216848FBF7A1FA1DE0644951
S31508007A704868FF21F531F9F74DFFC007C00F002808
S31508007A800ED180210920C006FBF791FA10210920A2
S31508007A90C006FBF78CFA01215B48FBF788FA04E07D
S31508007AA010210920C006FBF784FAFAF799FE7E2012
S31508007AB0FDF7BEF89CE0FAF7E9FDFBF773FD002336
S31508007AC001221946184600F099FA00231A46194663
S31508007AD0184600F093FA4A4840684A49884204D949
S31508007AE008214948FBF763FA1DE045494868FF2124
S31508007AF0F531F9F70FFFC007C00F00280ED1802116
S31508007B000920C006FBF753FA10210920C006FBF727
S31508007B104EFA01213C48FBF74AFA04E010210920F5
S31508007B20C006FBF746FAFEF793FB7E20FDF780F8C2
S31508007B305EE0FDF7D7FA20210920C006FBF739FADF
S31508007B40FAF7A4FDFFF768FEFDF7DEFEFBF72AFD50
S31508007B507E20FDF76DF84BE0FDF758FC2021092043
S31508007B60C006FBF726FAFAF791FDFFF755FEFDF773
S31508007B70CBFEFBF717FD7E20FDF75AF838E0FDF738
S31508007B80B1FA20210920C006FBF713FAFAF77EFDA1
S31508007B90FFF742FEFDF7B8FEFBF704FD7E20FDF772
S31508007BA047F825E0FDF732FC20210920C006FBF73F
S31508007BB000FAFAF76BFDFFF72FFEFDF7A5FEFBF7B8
S31508007BC0F1FC7E20FDF734F812E0FDF7B1FD202127
S31508007BD00920C006FBF7EDF9FAF758FDFFF71CFE7A
S31508007BE0FDF792FEFBF7DEFC7E20FDF721F800BFCD
S31508007BF000BF0EE700240140EC030020DA02000073
S31508007C000C020020204E000000040048FEB546483D
S31508007C100088FAF73EF90746444881693846FAF774
S31508007C20F1F900D2FEBD414A11685068F9F711FF13
S31508007C303E4988600A46D1689068F9F70AFF0290BB
S31508007C403A48C16801208007F9F70BFF00903748CA
S31508007C5081680098F9F701FF0746344801693846F4
S31508007C60F9F7A6FE0446314948690299F9F7F9FE7B
S31508007C7001902E4A91695069F9F7F3FE07462B4899
S31508007C80C1693846F9F72AFF054628488168284613
S31508007C90F9F7E7FE0546254A116A5069F9F7E1FE44
S31508007CA00746224881693846F9F718FF06462146ED
S31508007CB03046F9F7D6FE064629460198F9F778FEC2
S31508007CC007463146F9F774FE184948622A20085EC5
S31508007CD0FAF7D4F800901548416A0098F9F768FE53
S31508007CE00746FAF7FFF800B2104948852A20085EC9
S31508007CF0898D884204DD0D48808D00B20B49488580
S31508007D000A482A21415E002902DA002007494885E7
S31508007D100648C0680549086108468068C8600020AA
S31508007D200149088000BF7DE7500100203C0400207F
S31508007D3010B540210F48F9F730FE40210D48FAF7F3
S31508007D4021FF06210B48FDF7B9F90A4989898842B6
S31508007D500AD108482838008D0749884208D0FFF715
S31508007D6013FDFCF785FF03E0FFF70EFDFCF780FF28
S31508007D7010BD000074030020FBAA0000F7B5A0B0F0
S31508007D800C46154680216846F9F707FE00270026A7
S31508007D907E2168460170FE214170EF21817007211E
S31508007DA0C170209901710021417184712112C1713C
S31508007DB001210172457229128172012605E0684681
S31508007DC0805DC019C7B2701CC6B20B2EF7DBF8432C
S31508007DD0401CC1B26846C1727E2101730D21FCF7B1
S31508007DE06FFC23B0F0BDFFB5A1B006461C462A9F1E
S31508007DF0802101A8F9F7D1FD0020009000257E21F9
S31508007E00684601714671229981710721C1712399CA
S31508007E1001720021417284722112C172012101731B
S31508007E20477339128173012507E001A8415D00985F
S31508007E300818C0B20090681CC5B20B2DF5DB009877
S31508007E40C043401CC1B26846C1737E2101740D212E
S31508007E5001A8FCF735FC25B0F0BDFFB585B0054691
S31508007E600E460E9F00200190029003900490009009
S31508007E7000247E2168460171457186710421C1710D
S31508007E80079901720899417287723912C1720124E1
S31508007E9007E001A8015D00980818C0B20090601CB0
S31508007EA0C4B2082CF5DB0098C043401CC1B2684632
S31508007EB001737E2141730A2101A8FCF701FC09B070
S31508007EC0F0BDF7B584B005460E4600200090019037
S31508007ED002900390002700247E21684601704670B0
S31508007EE085700121C170694606980871012405E06C
S31508007EF06846005DC019C7B2601CC4B2052CF7DB22
S31508007F00F843401CC1B2684641717E218171072140
S31508007F10FCF7D6FB07B0F0BD70B504460D467E20CB
S31508007F20FCF786FE03E02078641CFCF7B9FB2846BC
S31508007F30691E8DB20028F6D170BD000030B5A1B01B
S31508007F400446802101A8F9F728FD0025002C02D057
S31508007F50012C20D10FE07E21684601710021417174
S31508007F60442181711321C1711522104902A8F9F71C
S31508007F70FBFC192510E07E2168460171FE2141713E
S31508007F80442181713321C1713622094902A8F9F7C2
S31508007F90EBFC3A2500E000BF00BF802D03DA294636
S31508007FA001A8FFF7B9FF21B030BD0000A6010020E7
S31508007FB0BB010020F8B506460C46FAF73BF9051E44
S31508007FC00F4600D00120014349000B484908411AD1
S31508007FD0C90F0DD0002E01D0012100E000210C436D
S31508007FE061004908401AC00F02D10120FCF7F2FED1
S31508007FF028463946F8BD00000000F07F0FB591B05D
S31508008000002010900F900E900D900C90FB48007871
S31508008010642803D0FA48C07F642803D10121F848B0
S31508008020017002E00021F64801701398002802D07A
S3150800803001287DD15DE2F348C1891298814203D1B6
S31508008040F048C08A0F9001E005200F900F98052888
S3150800805002DC05200F9004E00F98322801DB05208A
S315080080600F900F991298411A1198814217DDE4482A
S31508008070C078002859D1E34868384068E14968392A
S31508008080C8611498012803D10121DD48C1704CE06C
S315080080901498002849D10021D948C17045E00F99A4
S315080080A012984118119881423FDCD548C0780128BA
S315080080B03BD1D3482030407801282FD1D1486838A1
S315080080C04068D0496839C969401ACF4988420DD2F3
S315080080D0CB4898380089462820DDC9489838008951
S315080080E0801E81B2C6489838018117E0C5486838AD
S315080080F04068C4496839C969401A7D21890188429E
S315080081000CD9BF48983800895F2807DABC489838E0
S315080081100089801C81B2BA48983801810121B84883
S315080081202030417000212038C170B548C07800E081
S31508008130FDE301287ED1B2482030807B042804D094
S31508008140AF482030807B052804D10022012108464B
S31508008150FEF776F90F991298411A119881426ADD4D
S31508008160A848683840687D21C900884206D264203C
S31508008170A24908700021A2488171B3E1A04880791C
S3150800818000286CD101219E4881719E488089642807
S315080081905CDA9B484038018D408E081A81B29848AF
S315080081A040388186808E0990F9F773FE01460A9059
S315080081B096480068F9F792FC0B90F9F7DFFE944AA7
S315080081C003C28F484038008F40430990F9F768FE8C
S315080081D00B910A908E480CC80A98F9F76FFD8C4ADD
S315080081E003C28B4903C9FFF7E5FE0B910A90F9F71D
S315080081F0EDFE8849086082484038008F0890F9F7F4
S3150800820048FE0146099083480068F9F767FC8249E9
S315080082100A90F9F726FC0B90F9F77DFE7F4908705E
S315080082200846007864280DDC78480068F9F7A6FE49
S31508008230002201E053E16BE0794B0B910A90F9F7C4
S31508008240B1FE06D864207549087002E064207349B7
S3150800825008706B484038018D4030C18142E1694859
S315080082606838806C7D21C90088424CD90020654950
S31508008270683988646948007864283FDA6048403875
S31508008280018D4030C089814233DD012189075F486D
S315080082900068F9F78DFB0B90F9F73DFE81B2584857
S315080082A04038028D4030C089101A814205DA5B4891
S315080082B00078801E5949087020E051484038018DE1
S315080082C04030C089081A0A90F9F7D8FD0B904F4834
S315080082D001680B98F9F796FE10D250480078801C72
S315080082E04E49087008460078642807DD642008703F
S315080082F004E04A480078401D48490870404840381C
S31508008300018D4030C181454800783C490870E9E054
S315080083103B482030407800286ED13A488089642846
S3150800832003DB642035490870DCE036486838406865
S315080083307D21C900884206D2642030490870002190
S315080083402F488171CEE02E488079002872D101210C
S315080083502B4881712B488089642863DA284840387D
S31508008360018D408E081A81B2254840388186808E54
S315080083700990F9F78EFD01460A9024480068F9F736
S31508008380ADFB0B90F9F7FAFD214A03C21C484038A9
S31508008390008F40430990F9F783FD0B910A901C481A
S315080083A00CC80A98F9F78AFC194A03C2184903C97E
S315080083B0FFF700FE0B910A90F9F708FE15490860C9
S315080083C00F484038008F0890F9F763FD0146099079
S315080083D010480068F9F782FB0F490A90F9F741FB44
S315080083E00B90F9F798FD0D4908700846007864283F
S315080083F01BDD6420087018E06BE01BE0F20000202B
S315080084000C0400207402002070170000D40000201D
S31508008410D8000020E00000200000C842F10000203B
S315080084200000F03F6420FE490870FE48018D403088
S31508008430C18157E0FC48806C7D21C900884243D938
S315080084400020F9498864F748018D4030C089814287
S3150800845031DD01218907F5480068F9F7A9FA0B907B
S31508008460F9F759FD81B2EF48028D4030C089101ADC
S31508008470814205DAEA480078801EE94908701FE05B
S31508008480E848018D4030C089081A0A90F9F7F6FCC9
S315080084900B90E64801680B98F9F7B4FD10D2E0484E
S315080084A00078801CDE49087008460078642807DDD5
S315080084B06420087004E0DA480078401DD84908703E
S315080084C0D848018D4030C181D5480078D849087010
S315080084D008E0D4485838007AD549087002E00020E8
S315080084E0D3490870D248027814991398FDF7A8FF63
S315080084F01DE2CC486030807B012804D002287DD05C
S3150800850003287CD198E0C84868304188129881428F
S3150800851004D1C5486830408A0F9001E00A200F90C0
S31508008520C14840687D21C900884276D3BD4840309D
S315080085304079002871D1BB48018F403081820121E2
S315080085404171808A0A90F9F7A4FCBA490B90F9F7A9
S3150800855059FD1AD8B3484030808A0790F9F799FC34
S3150800856001460890B448F9F7B9FAB4490990F9F7F9
S3150800857078FAB3490A90F9F71BFA0B90F9F7CBFC8E
S31508008580C1B2A848603001703EE0A6484030808AF3
S31508008590FF210A31884219DCA2484030808A0790B8
S315080085A0F9F777FC01460890A248F9F797FAA34924
S315080085B00990F9F756FAA2490A90F9F7F9F90B90D2
S315080085C0F9F7A9FC9749603108701DE095484030D5
S315080085D0808A0790F9F75DFC014608909548F9F7F7
S315080085E07DFA98490990F9F73CFA95490A90F9F7FE
S315080085F0DFF90B90F9F78FFCC1B202E00EE029E033
S315080086000BE088486030017086486030007864283E
S3150800861003DB642083496031087029E082486830AA
S3150800862041881298814204D17F486830408A0F9069
S3150800863001E00A200F901BE07B4868308188129879
S31508008640814204D178486830808A0F9001E00A2078
S315080086500F900DE07448683081881298814204D1E1
S3150800866071486830808A0F9001E00A200F9000BF99
S3150800867000BF0F98052802DC05200F9004E00F982C
S31508008680322801DB32200F90664860308078002857
S3150800869002D11198FDF776FE0F991298411A119892
S315080086A0814221DB604840685F4908620020886390
S315080086B0C8635C491198C886084640300079002886
S315080086C00DD11498012806D11E21564840308177CD
S315080086D00121017103E00021524840300171002157
S315080086E050484030417041E10F991298411811984D
S315080086F08142F8DC4B4840300079012809D1002135
S315080087004848403001714848406847490862002097
S3150800871088634448603080780028E4D1424868304D
S31508008720408A0A280BDB4048406A0A90F9F7B1FBF1
S3150800873045490B90F9F7D2F94449086020E03A48D0
S315080087406830408A0A2810DA37486830408A07288D
S315080087500BDD3548406A0A90F9F79BFB3C490B90BC
S31508008760F9F7BCF9394908600AE02F48406A0A90C7
S31508008770F9F78FFB37490B90F9F7B0F933490860D9
S3150800878028484030008A0890F9F783FB0A90254864
S315080087904030008A0790F9F77CFB08902B4801685F
S315080087A00898F9F75EF909900A99F9F75AF90B90BA
S315080087B0F9F7E4FB284A03C21A4860300078401DDE
S315080087C00590F9F76DFB0991089016484030008A24
S315080087D00190F9F779FB059104901F4903C9FFF742
S315080087E0E9FB03910290059B049AF9F7CFFA0791E2
S315080087F00690099B089AF9F761FA0B910A90F9F71E
S315080088009FFB81B20748583881800748806A0A90DA
S31508008810F9F73FFB0E490B90F9F760F90B491DE094
S31508008820F1000020CC0300200C020020D400002018
S31508008830F200002000007A43000082430000BE4296
S31508008840000040400000B44200803B45CC000020B8
S315080088500000FA440080BB44E80000200860FB489A
S31508008860408A0890F9F715FB0A90F848408A07905D
S31508008870F9F70FFB0890F64801680898F9F7F1F838
S3150800888009900A99F9F7EDF80B90F9F777FBF14A91
S3150800889003C2EE4820300078401D0590F9F700FB2A
S315080088A009910890E948408A0190F9F70DFB05916E
S315080088B00490E84903C9FFF77DFB03910290059BE5
S315080088C0049AF9F763FA07910690099B089AF9F74B
S315080088D0F5F90B910A90F9F733FB81B2DB48983822
S315080088E0C180FF3801388089642829DADA48808906
S315080088F00890F9F7CEFA0A90D7486838406B059081
S31508008900F9F7C7FAD5490690F9F7E8F80890D24872
S315080089104188FF305930008E081A0690F9F7AEFAEA
S3150800892007900899F9F7DAF809900A9900E008E239
S31508008930F9F797F8CA490B90F9F7D0F8C9490860CA
S31508008940C24898388088642803DB6421BF48983871
S315080089508180BE489838C088642803DB6421BB48F8
S315080089609838C1800120B94920318870B748007904
S3150800897000287DD001287CD1B448807FBA4909787F
S3150800898088420BDA0021B148817701710020B2498B
S315080089906839C8640021AD48C17774E10F99129807
S315080089A0411A1198814210DDA8484079012805D15D
S315080089B0A648203001782038C17702E06421A34810
S315080089C0C1770121A14801705DE1A0482030807B74
S315080089D00300FCF7A4F906FD040A9CFCFBFD9B4872
S315080089E0203001782038C1774CE19B486838806B85
S315080089F099496839C96B401A7D21C900884256D9F8
S31508008A0095486838806B94496839C8638F484038F8
S31508008A10C18E119881420FDD8C48983880880A30BB
S31508008A2081B28A4898388180C08864283BDB6421F3
S31508008A3086489838C18036E00F980B9083484038AE
S31508008A40C18E1198411A0B98C20F10184010401C7D
S31508008A50814212DA7D4898388088801C81B27B482A
S31508008A6098388180C08864281DDB6421774801E036
S31508008A700AE14AE19838C18015E00F980B907348CF
S31508008A804038C18E1198411A0B98C20F1018401021
S31508008A90801C814207DD6D4898388088801E81B227
S31508008AA06A4898388180694940391198C8866A4861
S31508008AB06838406868496839096A401A6B498842C3
S31508008AC014DD624898388088401D81B25F4898381E
S31508008AD081808088642803DB64215C48983881801B
S31508008AE05D48683840685C496839086257482030EC
S31508008AF08078002805D15548203001782038C1777C
S31508008B0004E05248983801799830C177BAE052485B
S31508008B106838806B50496839C96B401A7D21C9008D
S31508008B20884257D94C486838806B4B496839C863BE
S31508008B3046484038C18E119881420FDD434898381F
S31508008B40C0880A3081B241489838C180C0886428F4
S31508008B5038DB64213D489838C18033E00F980B9084
S31508008B603A484038C18E1198411A0B98C20F10180E
S31508008B704010401C81420FDA34489838C088801C5F
S31508008B8081B232489838C180C08864281ADB6421CB
S31508008B902E489838C18015E00F980B902B4840381E
S31508008BA0C18E1198411A0B98C20F10184010801CDC
S31508008BB0814207DD25489838C088801E81B223483F
S31508008BC09838C18021494039119802E034E026E0FE
S31508008BD054E0C8862048683840681F496839096AD9
S31508008BE0401A2349884214DD18489838C088401D21
S31508008BF081B216489838C180C088642803DB64218E
S31508008C0012489838C180144868384068124968394B
S31508008C1008620E48983881799830C17732E00B4857
S31508008C20C078012804D100210848C177817702E07D
S31508008C301E210648C17700BF0448C078012819D10B
S31508008C4000210248C177817717E000000C04002054
S31508008C50CC000020E80000207402002000007A44BE
S31508008C600000C842D4000020F2000020881300004B
S31508008C70581B00001E213548C17700BF32213348F2
S31508008C80C17700BF00BF44E030482030807B012810
S31508008C9029D10F9912984118119881421FDB2B4848
S31508008CA0983801799830C1770F9912984018801E24
S31508008CB0119988420FDD26480078002824D12348D8
S31508008CC098388088401D81B22048983881800120D4
S31508008CD01F49087018E000201D49087014E000219B
S31508008CE01A48C17710E019482030807B042804D040
S31508008CF016482030807B052803D100211348C17708
S31508008D0002E00A211148C17703E000210F48C17724
S31508008D1000BF00BF0D482030807B012808D10B48D2
S31508008D20C07F02460B9014991398FDF789FB07E05C
S31508008D300648807F02460B9014991398FDF780FB2E
S31508008D4000BF00BF109815B000BD00000C0400203D
S31508008D50F000002010B5002201210846FDF770FB3F
S31508008D604C49088BF9F795F84B490860FEF74EFF12
S31508008D7048482030C079002839D1484846494860D3
S31508008D804448008BB42807D04248008BB32803D048
S31508008D904048008BB52804D101203E49203148724D
S31508008DA003E000203B49203148723D48406E3D496A
S31508008DB0884267D93748408B801E3B4909888842D4
S31508008DC00DDC3448408B801C37490988884206DB0D
S31508008DD0FEF716F901202F492031C87103E02D4806
S31508008DE0408B3149088000202D4948664AE02948C9
S31508008DF02030C07901283BD12C48274948602548AE
S31508008E00008BE62809D02348008BFF212C318842A5
S31508008E1003D02048008BE72804D101211D482030C3
S31508008E20417203E000201B49203148721C48406EFD
S31508008E301C49884226D91748408B801E1A4909883A
S31508008E4088420DDC1348408B801C174909888842E4
S31508008E5006DBFEF705FA02200E492031C87103E049
S31508008E600C48408B1049088000200D49486609E0E7
S31508008E7000200B494866084948850122FE215720EB
S31508008E80FFF71FF80448408DC2B201210020FDF704
S31508008E90D7FA10BD0C0400203C040020000034431F
S31508008EA00C02002088130000000100200000664321
S31508008EB030B503465A480068181AFF24F534A0420C
S31508008EC001D957480360481E904248DD5548007846
S31508008ED0002816D1881A3C2805DA881A3C24201A54
S31508008EE0514C207002E000204F4C20704E4800780C
S31508008EF05524201A4C4C2070204600784B4C207084
S31508008F002AE04B480078002822D14A480088401AAF
S31508008F1007280ADD454C2078C40F24186410424DF2
S31508008F202C7028460078414C207042480088401A28
S31508008F30012808DD3D480078401E3C4C207020463C
S31508008F400078394C20703B4802800120384C20704C
S31508008F5036480078344C2070364802805DE0481E5A
S31508008F6090424CDC481C824249DC2E480078012895
S31508008F7028D12F48007800282AD12E480088801A40
S31508008F8007280BDD294C2078C40F24186410264DB9
S31508008F902C7028460078254C20700DE0254800885E
S31508008FA0801A012808DB21480078401E1F4C2070D3
S31508008FB0204600781C4C20701E48028001201C4C5C
S31508008FC0207005E017480078002801D1164C20705B
S31508008FD0481E904205D115480078401E124C207054
S31508008FE01BE08A4205D111480078001F0E4C2070FC
S31508008FF013E00E480078801F0B4C20700DE000200F
S31508009000094C20700A4C20700120064C2070094833
S315080090100088824201DB074802800348007830BD99
S3150800902004010020F80000200201002003010020AE
S315080090300A0100200801002010B5FDF749FC0128A7
S3150800904000D110BDF748407F00287DD110210920A6
S31508009050C006F9F7ACFF80210920C006F9F7A7FF7B
S315080090600121F148F9F7A3FF0021EE48403081734A
S315080090700023012219461846FEF7C0FF00231A46A8
S3150800908019461846FEF7BAFFE8484068FF21F53149
S31508009090884209D2E3484030007B002803D10421E6
S315080090A0E148F9F786FFD6E20421DF48F9F77FFFA2
S315080090B00020DC4940310873DC484068DC498842B6
S315080090C0F1D9D8482030807800281CD120210920E1
S315080090D0C006F9F76CFFD54840687D2149018842EA
S315080090E001D2FBF78FFB0821CF48F9F760FF002173
S315080090F0CC48C1770020CB49403148708870CB49AD
S315080091004862486316E04021C748F9F747FF002838
S3150800911010D00021C348C1770020C24940314870A9
S315080091208870C24948624863BE4940318873012144
S31508009130BC4841774021BC48F9F730FF00280DD0DC
S3150800914020210920C00600E00DE0F9F732FF0020D3
S31508009150B449403188730121B24841777D204001E6
S31508009160B249486077E2AF484030807B0300FBF79E
S31508009170D6FD070571D8FEFDFCFB70000020A94945
S315080091804031087320210920C006F9F712FF002094
S31508009190A449403148708870A44948624863002150
S315080091A0A048203041710023012219461846FEF7CF
S315080091B025FF00231A4619461846FEF71FFF994849
S315080091C02038418D0186418D8185018DC18597485D
S315080091D040687D210901884228D9002095490870F0
S315080091E0904820308078002802D19049486002E0F3
S315080091F091488E49486040218B48F9F7CFFE0028F0
S315080092000CD1FBF7FFFA08218748F9F7D0FE7E2034
S31508009210FBF70EFD1E20F9F78FFB02E000208349BD
S31508009220486004218048F9F7C2FE12E008217E480A
S31508009230F9F7BFFE7D484068FF21F531884208D915
S31508009240784878384089002803D104217648F9F708
S31508009250AEFEFFE175484068FF21F531884204D229
S3150800926004217148F9F7A5FE03E004216E48F9F7D1
S315080092709EFE6E4948687D21C900F8F74BFB2328F6
S315080092802ED26A4948687D21C900F8F743FB192898
S3150800929026D964482038018DFF38593840888142DC
S315080092A007DA60482038418DFF38593840888142AE
S315080092B00DDB5C4840308078012821D100205B49CD
S315080092C048600862022057494031887318E0002038
S315080092D056494860086202215248403081730FE0BF
S315080092E0524948687D21C900F8F714FB232807D39B
S315080092F000204E494860086202214A48403081737E
S315080093004A4A68325188FF325932508D01231A462B
S31508009310FEF774FE00231A4619461846FEF76EFE37
S3150800932098E142484068FF21F531884204D2042179
S315080093303D48F9F73EFE03E004213B48F9F737FEBE
S315080093403A484168683000897D22D20050438142FC
S3150800935015D2364A68325188FF325932508D012368
S315080093601A46FEF74BFE03E01FE1B1E066E015E0A2
S3150800937000231A4619461846FEF740FE0DE000215E
S3150800938028482030017100202849486001212548D5
S31508009390203041700321203081735BE12148203859
S315080093A0408DFF217D31884204DC1E482038008D1F
S315080093B088420CDD0023012219461846FEF71EFED8
S315080093C000231A4619461846FEF718FE29E01749DB
S315080093D048687D21C900F8F79DFA1449683149891A
S315080093E0884210D2114A68329188FF325932508D1C
S315080093F001231A46FEF702FE00231A4619461846A6
S31508009400FEF7FCFD0DE007482038018D4186002057
S3150800941006494860002103482030017104212030A4
S31508009420817317E1EC030020000400480C020020B9
S31508009430B80B0000C4000020C40900008848408D0D
S31508009440FF217D31884203DC8548008D88420CDD8A
S315080094500023012219461846FEF7D0FD00231A46B6
S3150800946019461846FEF7CAFD31E07E4948687D214F
S31508009470C900F8F74FFA7B496831098A0F398842DB
S315080094801ED2784A6832D189754A108D0123002286
S31508009490FEF7B4FD72484030C078012806D1002393
S315080094A0012219461846FEF7A9FD10E06D4A6832F2
S315080094B0D1886B4A508D01231A46FEF79FFD06E0B8
S315080094C00020684948600520654960318873C1E015
S315080094D064484068FF21F531884204D20421624875
S315080094E0F9F767FD0FE05F484068FF21F5318842CC
S315080094F009D95C4840684B21C900884203D2042137
S315080095005948F9F754FD57484068584988421ED2C9
S31508009510544A6832D189524A108D01230022FEF737
S315080095206DFD4F484030C078012806D1002301223E
S3150800953019461846FEF762FD36E04A4A6832D1886F
S31508009540474A508D01231A46FEF758FD2CE00421A0
S315080095504548F9F72EFD434840684449C8318842D2
S3150800956022D300203F4948603D486030C07A012830
S3150800957004D106203A496031887305E0002138484D
S315080095806030817340384177002301221946184616
S31508009590FEF734FD00231A4619461846FEF72EFD37
S315080095A004213148F9F703FD54E000212C484030E6
S315080095B00171C17000202B490865C864002128483C
S315080095C06030017320210920C006F9F7F2FC00215A
S315080095D02348603041708170002022494862486300
S315080095E000211F48403041710023012219461846C0
S315080095F0FEF704FD00231A4619461846FEF7FEFC38
S315080096001748418D0186418D8185018DC1852030A0
S31508009610C07F00281DD1134840681549884218D9CB
S31508009620FBF7F0F800200F4948600D485838408885
S31508009630032808DA0A48408D82280ADC01200849EE
S315080096406031887305E00021054860308173403831
S31508009650417700BF00BF7E20FBF7EAFA00BFF0E4BF
S31508009660CC0300200C02002000040048A4380000A7
S3150800967060EA000094960008C80000204401000033
S31508009680FC220008E49600080C020020940800005A
S31508009690C44D0008015E2D010203040435060708BF
S315080096A009ACA24A041A5916011129250A4501814D
S315080096B0580B1058594C4C3031313278010B11CBBC
S315080096C07E153E0401320505133812061459413237
S315080096D030303532384834353034324120041B7D39
S309080096E05D7E00009D
S705080018C515
